:020000040800F2
:10000000709C0020C1020008A9770008AB770008A7
:10001000BD770008BF770008C17700080000000026
:10002000000000000000000000000000D3020008F3
:10003000C377000800000000D70200081150000834
:10004000DB0200089B570008DB020008CF480008CD
:10005000DB020008DB02000881460008A146000818
:10006000C3460008E346000805470008774000083B
:10007000B9400008FB4000084741000893410008D0
:10008000AF420008FF420008DB020008DB02000864
:10009000DB020008DB020008DB020008254700083D
:1000A000DB020008DB020008DB020008DB020008BC
:1000B0005D5200087F520008A1520008DB020008D0
:1000C000DB020008DB020008DB020008DB0200089C
:1000D000DB0200083D3B0008AD3B00081D3C00086A
:1000E0006747000807490008DB020008DB02000838
:1000F000DB020008DB020008DB020008DB0200086C
:10010000DB020008DB020008C3520008DB02000823
:100110008D3C0008013D0008E55200080753000827
:100120004F4300089D430008ED4300083944000890
:1001300000F002F800F0B0F80AA090E8000C824449
:100140008344AAF10107DA4501D100F0A5F8AFF226
:10015000090EBAE80F0013F0010F18BFFB1A43F0A5
:1001600001031847F0C3000010C400000A444FF018
:10017000000C10F8013B13F0070408BF10F8014B06
:100180001D1108BF10F8015B641E05D010F8016B4B
:10019000641E01F8016BF9D113F0080F1EBF10F8AF
:1001A000014BAD1C0C1B09D16D1E58BF01F801CBD2
:1001B000FAD505E014F8016B01F8016B6D1EF9D555
:1001C0009142D6D37047000000230024002500266A
:1001D000103A28BF78C1FBD8520728BF30C148BFAA
:1001E0000B6070476E2907F0C185702907F0A7865C
:1001F00066290AF08B8265290AF0888267290AF04D
:10020000858261290AF0848203681B0A28BF41F0B5
:100210008001692907F06E85642907F06B857529CF
:1002200007F068856F2907F03586782907F073860F
:10023000E92908F06781E42908F06481F52908F0CC
:100240006181EF2907F03286F82907F0728603688A
:10025000DB0928BF41F08001632908F01E81732962
:1002600008F02381E32908F04181F32908F0468151
:10027000002070471FB508F061FE04000020002137
:1002800009F04CFD401C60600020002109F05CFD7D
:10029000E0601FBD10B510BD08F02BFE1146FFF742
:1002A000E9FF00F0BEF808F009FF03B4FFF7F2FF22
:1002B00003BC03F014FA000080F3088870470000C4
:1002C0000948804709480047FEE7FEE7FEE7FEE7EA
:1002D000FEE7FEE7FEE7FEE7FEE7FEE70448054926
:1002E000054A064B704700002978000831010008D4
:1002F000706C0020709C0020707C0020707C0020BE
:1003000070B502246E4D641E2878C00709D16DA017
:1003100000F0CFFC01F0FCFB03285ED06BA002F0E4
:1003200015FE2878C1071AD0800718D46AA000F0FB
:10033000C0FC1E2002F0CCFD06461E21304601F016
:1003400036FF032851D0287820F00100287001F0F2
:1003500091FC304602F0FAFD304602F0F3FD2878B9
:10036000C10711D081070FD540070DD45CA000F064
:10037000A0FC00F050FD03283CD0287820F00400B9
:1003800028705BA002F0E2FD2878C10711D0810738
:100390000FD5C0060DD459A000F08BFC00F0F8FC7E
:1003A000032833D0287820F01000287057A002F0DE
:1003B000CDFD002CA7DA2878C1072FD081072DD5D5
:1003C000C0062BD50324544801F0D9FE5248401FE3
:1003D00001F090FC00F04CFC21E0287840F0010096
:1003E00028704EA002F0B2FD9BE7287840F0020092
:1003F0002870AEE7287840F0040028704AA1422017
:1004000000F023FD4EA002F0A1FDBDE7287840F0EA
:10041000100028704DA002F099FDCCE70224204680
:1004200070BD10B54C4800F025FB4FF4407005F04E
:10043000BBF94A4800F025FA4FF4165000F0A2FE2E
:1004400000F01BF904F0AEFF01F062FB0222510242
:1004500043A002F0E3FB4048807800F0ABFD00F0E1
:1004600018F94FF0E020016921F0030101613E48D5
:10047000016841F0007101603C4C204600F0E9FD4C
:100480003B48006800F096FD00F003F9204600F0BC
:10049000E0FD2409204600F08DFD00F0FAF820462A
:1004A00000F0D7FD33A000F004FC35A000F00EFCF6
:1004B00042F2107004F0FCFD07F0AAF9002010BD14
:1004C00000000020CED5CAD6D6D03A00CED5CAD6A6
:1004D000CAA7B0DC00000000C8EBCDF8D6D03A00C7
:1004E000C1ACBDD3544350B7FECEF1C6F73A0000BD
:1004F000544350C1ACBDD3CAA7B0DC00C1ACBDD31E
:10050000465450B7FECEF1C6F73A0000465450C1EB
:10051000ACBDD3CAA7B0DC007C100020CED5CAD6B3
:10052000B3C9B9A60000000044657669636520740C
:10053000637020636F6E6E657463656421000000F4
:10054000544350C1ACBDD3B3C9B9A600465450C141
:10055000ACBDD3B3C9B9A60064070020F4060020DF
:10056000647373730000000004ED00E000001C8061
:1005700034070020C9E8B1B8B9CAD5CF3A000000A5
:10058000C7EBC1AACFB5B3A7BCD2000070B5054672
:100590000C467B2005F0E2FA012804D12246CAA1CC
:1005A000284607F0B4FE7C2005F0D8FA012804D1D3
:1005B0002246C8A1284607F0AAFE7D2005F0CEFA03
:1005C000012804D12246C6A1284607F0A0FE7E20BD
:1005D00005F0C4FA012804D12246C5A1284607F037
:1005E00096FE7C2005F0BAFA88B97D2005F0B6FAAF
:1005F00068B97E2005F0B2FA48B97A2005F0AEFA63
:10060000012804D12246BEA1284607F080FEBDE89D
:10061000704005F0CABB10B5BC48044604F0EEF8C3
:1006200022460B21BAA007F0DBFABE480022426046
:100630008260C2600B222146001D07F068FEB948A7
:1006400000F008FAB1480121253804F0E0F8AF4A7B
:100650001821253AB4A007F0C3FAAC480B210C309E
:100660000446FFF793FF22460B21B4A007F0B8FA27
:10067000BDE81040B64807F0B3BA10B504F0D4FC9A
:10068000002002F02DFFFFF7C6FFBDE8104004F088
:1006900089BE70B50324AF4D2978490704D5AEA0B3
:1006A00002F054FC00F0AEFB2978C90605D5AEA0D7
:1006B00002F04CFC00F082FB0446204670BD70B591
:1006C000044602250121201D04F0A1F8ABA1201D44
:1006D00007F07BFD211DAB4802F06BFA032813D015
:1006E0001D21201D07F0ECFDA7A1201D07F06DFDC9
:1006F000211DA94802F094FE002803DB012084F8A4
:1007000021000325284670BD002084F82100032520
:10071000F8E76FF30F00A149401804D0B0F5003F8F
:1007200003D0002070479E4870479E48704770B5C0
:1007300005460E460224A2020021281D02F06EFA90
:100740003060002807DB98494058FFF7E2FF286037
:1007500010B1032400E00424204670BD7CB504469B
:10076000022084F8290047E090A1CDE90010002381
:1007700003221021184600F0CEFE00F0E6FC6420B3
:1007800004F096FC4FF4006694F8290094F82810C1
:10079000884202D1A18CC1F30A06401EC102324632
:1007A000201D02F03BFA0546002D2DDB94F8292090
:1007B00081A1422000F049FB94F829002168401EE5
:1007C00001EBC02078493246091F294404F020FF7C
:1007D000032807D094F829207DA1422000F035FBA2
:1007E00004207CBD14F8292F86A1422000F02DFBA7
:1007F0002078401C04F8290994F8290094F828105E
:100800008842B1D903207CBD94F8292084A14220DC
:1008100000F01BFB02207CBD70B50546002406F0ED
:1008200092FC8B49681A8D4227D006DC312D24D0EA
:10083000322D09D0332D20D113E0B0F5003F03D085
:10084000B0F5802F19D10CE04025554E05E006EBA0
:10085000C42006F0B1FC641CE4B26D1EEDB2F6D209
:100860000BE040254F4E05E006EBC42006F0A4FC4B
:10087000641CE4B26D1EEDB2F6D2BDE8704006F025
:100880006EBC002140F8191F41608160C1600161A8
:1008900041611938192107F0F1BC10B504460B224B
:1008A00004F1190007F033FD002084F8250010BD85
:1008B00010B504460B2204F1250007F028FD0020A6
:1008C00084F8310010BD0000D6D8C9CFB5E7C6F412
:1008D000B6AF0000C8EDB8B4CEBBC6F4B6AF0000EA
:1008E000B6C0C1A2BFB4C3C5B9B7C6F4B6AF0000A5
:1008F000B4B0BFDABFB4C3C5B9B7C6F4B6AF000071
:10090000D3B2B8B4CEBBC6F4B6AF0000190700200E
:100910000D0A426F6F74B0E6B1BE203A20252E2A30
:1009200073000000640700200D0AC9E8B1B8B1E007
:10093000BAC5203A20252E2A730000000D0AD6D809
:10094000C6F4D4ADD2F2203A20252E2A730000003E
:1009500054C1000800000020424F4F54B6CFBFAA38
:10096000544350C1ACBDD300424F4F54D7A2CFFA2D
:10097000465450B5C7C2BD21000000002E62696E0A
:100980000000000018010020436F6D6D6F6E417014
:10099000702E62696E0000009A1000200000FDF7C2
:1009A00000C0030800C005081E130020CFC2D4D821
:1009B000D7D3B0FC3A256400D7D3B0FCA3BA2564E2
:1009C00020A1A3CFC2D4D8B3C9B9A6A3A100000067
:1009D000D7D3B0FCA3BA256420A1A3D0B4C8EB46FA
:1009E0004C415348CAA7B0DCA3A1C9E8B1B8BCB414
:1009F000BDABCCF8D7AAB5BDD3A6BCB1B3CCD0F2B1
:100A0000A3A10000D7D3B0FCA3BA256420A1A3D032
:100A1000B4C8EB464C415348B3C9B9A6A3A10000E2
:100A2000D7D3B0FCA3BA256420A1A3CFC2D4D8CA1F
:100A3000A7B0DCA3A1C9E8B1B8BCB4BDABCCF8D7B2
:100A4000AAB5BDD3A6BCB1B3CCD0F2A3A10000001F
:100A500000C001080146F822544804F048BD10B512
:100A6000F82107F00BFCBDE81040F82250494F4830
:100A700004F09ABC7CB504462046FFF7F0FF5B20EB
:100A800020706078FF2801D130206070A17831207B
:100A9000FF2900D1A070E178FF2900D1E070207C0F
:100AA00004F11005FF283DD02946424800F03AF9EC
:100AB00094F8500004F15005FF283CD029463D48E9
:100AC00000F03EF994F8900004F19005FF283BD027
:100AD0002946384800F041F994F8D00004F1D005D7
:100AE000FF283BD02946334800F044F994F8E00051
:100AF000FF283CD088B32E492F48E03100F06EF932
:100B000094F8F000FF283DD000283BD028492A481F
:100B1000F03100F070F95D2084F8F7002046BDE860
:100B20007C4097E74021284607F0A8FB23A12846F0
:100B300007F0FDFABCE74021284607F09FFB21A102
:100B4000284607F0F4FABDE74021284607F096FB57
:100B50001DA1284607F0EBFABEE708E01021284661
:100B600007F08CFB1CA1284607F0E1FABEE704F170
:100B7000E0001021054607F081FB17A1284607F089
:100B8000D6FABDE70020C4F8F000A4F8F400009005
:100B900001900A22694641F6583002F0CAFB6946C4
:100BA00004F1F00007F0C3FAB5E70000008801087F
:100BB00064070020020000209A0100202F41424DCE
:100BC0000000000041424D0053686F7033343437E9
:100BD00039343734390000003132312E352E32317C
:100BE000372E32353200000008B5002300901A4637
:100BF0001021184600F08FFC08BD1CB504461021DA
:100C0000002200913EA31146104600F059FC3F49D6
:100C10000022CDE90021002110232022084600F007
:100C200046FE0C2100220091234611461A2000F0B6
:100C300047FC1CBD1CB5044610210022009130A3C6
:100C40001146402000F03CFC304900224031CDE903
:100C50000021102320220021402000F028FE0C213A
:100C600000220091234611465A2000F029FC1CBDA9
:100C700010B5102002F02CF90446254B25A21021B6
:100C8000204606F0B9FF2046FFF7D4FF102120468A
:100C900007F0F4FA1E4B21A25B1D1021204606F03E
:100CA000ABFF2046FFF7A9FF2046BDE8104002F049
:100CB00049B908B50023009001221021184600F020
:100CC0002AFCBDE80840022000F01ABC08B5002349
:100CD000009002221021012000F01DFC08BD38B553
:100CE0000C460023009001221021184600F013FC4E
:100CF0000023022210211846009400F00CFC38BD9D
:100D000020202020202020200000000004A800082F
:100D10007710002025736D560000000043535125C5
:100D20007300000070B50C4600F58B7080210546FD
:100D300007F0A4FA21462846BDE8704007F0F7B94D
:100D400070B504460D468021601C07F097FA2946CD
:100D5000601CBDE8704007F0EAB970B50C46813000
:100D60008021054607F08AFA21462846BDE87040F2
:100D700007F0DDB970B50C4600F58270102105460C
:100D800007F07CFA21462846BDE8704007F0CFB94D
:100D900010B5114801F073FE03280ED10E4801F082
:100DA0009CFE032809D10C4801F0B6FE032804D1AB
:100DB000BDE81040084801F0DDBE10BD10B5064882
:100DC00001F0D5FE032805D103480078BDE81040A6
:100DD00001F0FBB810BD00000200002070B5044611
:100DE0000D461021601C07F049FA2946601CBDE839
:100DF000704007F09CB910B50446084607F06EF93C
:100E0000608210BD10B5002001F040FCBDE810402C
:100E1000012001F0DAB810B501F062FB03280CD113
:100E2000444801F037FC04464249032C06D04A8A64
:100E3000491C41A002F0E4F8204610BD4A8A491C32
:100E400044A002F083F8204610BD0FB4F8B5064662
:100E5000022540F2492002F03BF8044608AB00931B
:100E60002F02394604F12600079A06F09FFE00285B
:100E700001DDB8420BDD82223DA142A002F0C0F8A4
:100E8000204602F05FF80220F8BC5DF814FB28222F
:100E900022706670642290FBF2F13031A17090FBF9
:100EA000F2F102FB11010A2291FBF2F13031E17003
:100EB00090FBF2F102FB1100303020711D49891EB8
:100EC00008786071401CC0B20870392801D9302000
:100ED0000870042232A1A01D07F019FA012104F1C3
:100EE0000A0003F094FC3B2184F8221030220221F6
:100EF00004F1230007F0BAF9262184F82510032213
:100F000029A1204607F001F929480078400708D5B3
:100F1000204607F03BF982B22146064801F0CFFB9C
:100F20000546204602F012F8204602F00BF828464B
:100F3000AAE700009A0100205443502053657276BE
:100F40006572C1ACBDD3CAA7B0DC3A25733A25643B
:100F500020A3A10054435020536572766572C1AC42
:100F6000BDD3B3C9B9A63A25733A256420A3A1001D
:100F7000555345525F5443505C757365725F74639B
:100F8000702E630025732C25643A7570446174617A
:100F9000427566207370696C6C6F766572A3A100F0
:100FA0004D41433A000000002458290D0A0000007A
:100FB0000000002070B50446002504F0F3F92E4E21
:100FC000A01BB44211D006DC312C0ED0322C1DD027
:100FD000332C06D12BE0B0F5003F17D0B0F5802FB1
:100FE00025D026A14220FFF730FF706840F60101AE
:100FF000B1EB104F05D12AA14220FFF726FF35465D
:1010000020E02DA14220FFF720FF1BE0304C60685C
:101010002114B1EB104F05D12EA14220FFF715FF8F
:1010200025460FE031A14220FFF70FFFDDE7354CE9
:1010300060682114B1EB104F06D133A14220FFF7B5
:1010400004FF2546284670BD35A14220FFF7FDFE6E
:10105000CBE710B50168384A1140B1F1005F09D102
:101060004168364C21600068FFF726F92068BDE82A
:101070001040004710BD000000C001084150504E14
:10108000554DB2BBBACFB7A8A3A1BCB4BDABD6B4C3
:10109000D0D0D3A6BCB1B3CCD0F2A3A10000000045
:1010A000BFAACABCD6B4D0D041505031D3C3BBA71D
:1010B000B4FAC2EB2100000041505031D3C3BBA7AA
:1010C000B4FAC2EBD2D1CADCCBF0A3A1000000007D
:1010D00000C00308BFAACABCD6B4D0D04150503219
:1010E000D3C3BBA7B4FAC2EB210000004150503279
:1010F000D3C3BBA7B4FAC2EBD2D1CADCCBF0A3A155
:101100000000000000C00508BFAACABCD6B4D0D0F9
:1011100041505033D3C3BBA7B4FAC2EB2100000047
:1011200041505033D3C3BBA7B4FAC2EBD2D1CADC0F
:10113000CBF0A3A1000000000000FE2FB0010020B2
:1011400010220921042003F0F9B90921042003F039
:101150005BBA10B5FFF7F9FF4FF4C87003F0A8FFB2
:10116000BDE81040F1E7000010B50A4601461148FD
:1011700001F0C9FF002804D0BDE810400EA001F026
:101180003FBF10BD10B504460A4801F0B3FF01236C
:101190000C222146022002F0ADFAAFF23301BDE885
:1011A0001040022002F07ABA0A460146022002F0FC
:1011B000D6BB00005C0800207355736251756575DD
:1011C00065D2E7B3F6A3A1000320401EC0B2FCD253
:1011D0007047F0B50346002500260127F94C012988
:1011E0000CD00022C4F89861C4F89061C4F89461EE
:1011F0003AB118060DD5C4F89C610CE0C4F898719A
:10120000F2E7180602D5C4F89C7104E0C4F89C61AA
:1012100001E0C4F89C71C4F89471FFF7D5FF58063B
:10122000030E6D1CEDB2082DE0D3C4F89071C4F824
:101230009871F0BD10B50446B031C8B20022114615
:10124000FFF7C7FFA41CC4F30310002240F01000F6
:101250001146FFF7BEFF04F00F000022BDE810406A
:101260001146B6E730B5002505F1B0000022C0B246
:101270001146FFF7AEFF002211460220FFF7A9FF3B
:10128000002211461020FFF7A4FF002400220121B4
:101290001046FFF79EFF641CE4B2802CF6D36D1C51
:1012A000EDB2082DE0D330BD70B51022042100202E
:1012B00003F044F910220521002003F03FF9102229
:1012C0000621002003F03AF910220721002003F044
:1012D00035F910220521022003F030F9BA4C01251E
:1012E0002560642003F0E4FE00202060642003F009
:1012F000DFFE256000221146AE20FFF76AFF0022C4
:1013000011460220FFF765FF002211461020FFF76B
:1013100060FF002211464020FFF75BFF00221146CC
:101320008120FFF756FF00221146FF20FFF751FFF3
:1013300000221146A120FFF74CFF00221146C820D1
:10134000FFF747FF00221146A620FFF742FF0022C9
:101350001146A820FFF73DFF002211463F20FFF76E
:1013600038FF00221146D320FFF733FF0022114639
:101370001046FFF72EFF00221146D520FFF729FF68
:10138000002211468020FFF724FF00221146D920B9
:10139000FFF71FFF00221146F120FFF71AFF00227E
:1013A0001146DA20FFF715FF002211461220FFF741
:1013B00010FF00221146DB20FFF70BFF0022114631
:1013C0004020FFF706FF002211462020FFF701FF13
:1013D000002211460220FFF7FCFE002211468D205C
:1013E000FFF7F7FE002211461420FFF7F2FE00225D
:1013F0001146A420FFF7EDFE00221146A620FFF7BC
:10140000E8FE00221146AF20FFF7E3FE002211465E
:10141000AF20FFF7DEFEFFF725FFBDE8704000219B
:10142000084607E72DE9F041804606980E461F461C
:1014300000242038C5B2B8F17F0F02D9A046B61CEF
:10144000F6B20C2A06D0102A19D0BDE8F0415FA0F0
:1014500001F0D6BD761CF1B24046FFF7EBFE6049C5
:1014600005EB450001EB40053A46285D0121FFF7F9
:10147000B0FE641CE4B2062CF6D3BDE8F081314620
:101480004046FFF7D7FE574800EB05153A46285D62
:101490000121FFF79EFE641CE4B2082CF6D3761CF3
:1014A000F1B24046FFF7C6FE002428193A46007AFA
:1014B0000121FFF78EFE641CE4B2082CF5D3DCE7B3
:1014C0002DE9F8430446DDF820800E4691461F467C
:1014D000002510E000904B46424631462046FFF77B
:1014E000A1FF04EB5800C4B2782C02D90024761C6A
:1014F000F6B26D1CEDB2785D0028EBD1BDE8F88343
:1015000008B5102140060091010E002236A31046B6
:10151000FFF7D6FF08BD0FB42DE9FE4F0C469346EA
:1015200000254FEA54088020B0FBF8F64FEA4B073D
:10153000102C1BD0042002900DF14409CDF804902A
:10154000701C01F0C5FC82464B46711C5046109A37
:1015500006F02CFB8146B1450BD90AEB060010F8CA
:10156000010C7F2805D9A6F1010905E0642002904D
:10157000E2E7B14500D9B1460C98012802D0022813
:101580000AD105E0A6EB0900400808FB00F503E0DE
:10159000A6EB090008FB00F5B9F1000F7DDD584608
:1015A000FFF7AEFF0026A8E01AF806107F2925D81D
:1015B0000091F9B2E8B222460F9BFFF733FF05EB2B
:1015C000540599E000002142940122424E6F2020F0
:1015D00043484152484947485F65202E00000000BB
:1015E0009CB60008C4B8000820202020202020201D
:1015F000202020202020202000000000002078E073
:10160000102C02D00C2C38D072E0C0EBC00202EBE0
:101610008203DA4A03EB020898F82020914267D14E
:101620000AEB060298F8213052789A4260D1F9B25A
:10163000E8B2FFF7FFFD4FF0000B07E018F80B00D2
:1016400001210F9AFFF7C5FD0BF1010BA345F5D35F
:10165000781CC1B2E8B2FFF7EDFDA34607E018F829
:101660000B0001210F9AFFF7B4FD0BF1010BBBEB4F
:10167000440FF4D32544761C3EE000EBC00202EB9D
:101680004203BE4A6C3A03EB020898F818209142D4
:101690002ED10AEB0602527800E032E098F81930B9
:1016A0009A4225D1F9B2E8B2FFF7C4FD4FF0000B22
:1016B00007E018F80B0001210F9AFFF78AFD0BF1E4
:1016C000010BA345F5D3781CC1B2E8B2FFF7B2FD18
:1016D000A34607E018F80B0001210F9AFFF779FDE8
:1016E0000BF1010BBBEB440FF4D32544761C03E054
:1016F000401C029A904283D3761C4E45FFF454AFAF
:1017000009E008D0B6229EA1A3A006F069FAAFF2C4
:10171000341006F065FA5046BDE8FE0F5DF814EB94
:1017200001F010BC00B5002211468D20FFF751FDDD
:10173000002211461420FFF74CFD00221146AF2075
:101740005DF804EB45E500B5002211468D20FFF75A
:1017500040FD002211461020FFF73BFD00221146FC
:10176000AE205DF804EB34E52DE9FF5F80460E9D69
:101770008B461F46002459464046FFF75BFD0BF1A0
:1017800001090C2D08D0102D4FD0AFF2C01004B0BD
:10179000BDE8F05F01F034BCDFF8E0A1AAF16C0A0B
:1017A0003CE06C221B2300203D1932E000EBC00618
:1017B00006EB46065644395D96F818C0614527D1B8
:1017C000697896F819C0614522D159464046FFF71D
:1017D00031FD00250121705D029AFFF7FAFC6D1CB6
:1017E000EDB20C2DF6D309F0FF014046FFF722FDC4
:1017F0000C250121705D029AFFF7EBFC6D1CEDB228
:10180000182DF6D308F10C0808F0FF08641C04E05A
:10181000401C92FBF3F18142C8D8641C384606F0A4
:10182000B5FCA042BDD8BDE8FF9FDFF850A138E06D
:1018300000203A5D3B19C0EBC00101EB810101EBD7
:101840000A0696F820108A4227D1597896F8215036
:10185000A94222D159464046FFF7ECFC0025012160
:10186000705D029AFFF7B5FC6D1CEDB2102DF6D33A
:1018700009F0FF014046FFF7DDFC10250121705DF6
:10188000029AFFF7A6FC6D1CEDB2202DF6D308F1ED
:10189000100808F0FF08641C02E0401C6428CAD34A
:1018A000641C384606F072FCA042C1D8BBE72DE9A3
:1018B000F04F8146DDE909BA0E460025580705D0EC
:1018C000012000EBD30702EB090815E0DF08FAE777
:1018D00031464846FFF7AEFC4C4609E028466D1CF1
:1018E0001AF800005A460121FFF773FC641CE4B2A9
:1018F000A045F3D8761CF6B2BE42E9D3BDE8F08F1E
:1019000010B586B00121080304F019FA042206215B
:10191000002002F013FE18220521002002F00EFE26
:1019200018220721002002F009FE102204210020C5
:1019300002F004FE0020ADF804004FF48271ADF80F
:101940000610ADF80800ADF80A00ADF80C004FF431
:101950000071ADF80E100821ADF81010ADF81200AE
:101960000720ADF81400104C01A9204605F0EEFF49
:101970000121204606F06FF806B010BDF0A800085F
:101980002E2E5C48415244574152455C4F4C4544D1
:101990005C6F6C65642E63004C6F674572723A2011
:1019A00025732C256400000000300140072813D265
:1019B000DFE800F00406080A0C0E1000D9A07047FA
:1019C000DAA07047DCA07047DEA07047E0A0704747
:1019D000E2A07047E4A07047E7A070474FF4A07101
:1019E000E84806F04BBC4FF4A071E74806F046BC4F
:1019F000E649002048604FF41061E54806F03EBC1F
:101A000070B506460D46E14C207800280AD0E04823
:101A100061682A460844314606F0E3FB60682844C2
:101A2000606070BDDBA1304601F0FAFC002821DBCC
:101A3000DAA1304601F0F4FC00280DDB2A463146DD
:101A4000DA4801F060FB0028EBD0BDE8704083224B
:101A5000D7A1E0A001F0D4BA2A463146E44801F00B
:101A600052FB0028DDD0BDE870408A22D0A1E1A061
:101A700001F0C6BAC34806F089FBC0F5A070A842C1
:101A800005D93146BDE87040BE4806F09EBB96229F
:101A9000C7A1DFA001F0B4FAFFF7A0FF3146BDE80F
:101AA00070404FF4A072B74806F031BCDF49002007
:101AB000086040F6B83003F0FBBA10B510220F21D1
:101AC000042002F03BFDFFF7F1FF10220B21042060
:101AD00002F034FDD54900201039086010BD10B562
:101AE00000230C224FF41651184601F003FEFFF7B5
:101AF00075FFFFF778FFAD4801F0FCFABC4801F034
:101B0000F9FAAFF20311BDE81040002001F0C6BDA4
:101B100010B50424FFF7E3FFFFF7CFFF204610BD09
:101B20000FB42DE9F84F82464FF004089748CAEBEE
:101B3000CA01083000EB8104667E60680B904FF4A8
:101B4000A165284601F0C4F983460CAB00932946F1
:101B500058460B9A06F02AF807464FF00009002F66
:101B600001DDAF423EDDC22291A1B1A001F048FAF1
:101B7000584601F0E7F90220BDE8F80F5DF814FBC4
:101B8000FFF72CFF0025BAB25946002001F0E7FE0E
:101B900016E0642003F08CFAE1687A4801F040FC1A
:101BA00020612069002802DB4FF003081DE0616915
:101BB000744801F035FC002802DB4FF0020814E005
:101BC00028466D1C2189EDB28842E2D3607E801BDD
:101BD00000EBC00101EB00104FF4FA7101EB800043
:101BE00003F066FA761EF6B2CAD2584601F0AAF998
:101BF000CDF80090B8F1050F0ED2DFE808F003052C
:101C000007090B0091A408E093A406E095A404E062
:101C100096A402E097A400E098A45046FFF7C6FE01
:101C20000146224698A001F0BFF94046A4E77F494B
:101C300001200860704770B500240425FFF7F7FF06
:101C4000FFF7CCFE4FF47A7610E0641CE4B2304625
:101C500003F02EFA8EA14B4801F0E2FB002805DBD1
:101C600021468CA001F0A0F9032501E0142CECD34F
:101C7000284670BD10B500210846FFF751FF044605
:101C8000032C02D089A001F0BBF94FF47A7003F065
:101C90000FFAFFF70BFF204610BD002101203FE7A0
:101CA00010B500210220FFF73BFF032808D00021D8
:101CB0000320FFF735FF0021BDE8104002202FE789
:101CC00010BD70B505461521284606F0D7FA00214B
:101CD0000520FFF725FF0446032C09D10D212948D3
:101CE00006F009FA811C14230D22284601F0BBFAE4
:101CF000204670BD70B50446002020602071002190
:101D00000620FFF70DFF0546032D09D12C211D48A4
:101D100006F031FA411C04230D22204601F0A3FAFB
:101D2000284670BD5455524E4F46460048414E44D9
:101D30005348414B450000005155455259434F4EC1
:101D400046494700434C4F534545434F0000000070
:101D500053415645434F4E46494700005155455261
:101D60005952454C455345005155455259564F4CD3
:101D70005441474500000000CEDEB4CBC3FCC1EEA9
:101D8000000000009A100020DA110020B4010020A9
:101D90001A1300202B51495552433A002B514955F3
:101DA00052433A2022726563762200001A1C0020FA
:101DB0002E2E5C48415244574152455C4C54455C80
:101DC000454332305C656332306D6F64756C652EEF
:101DD0006300000025732C25643A735463705175B9
:101DE000657565207370696C6C6F766572A3A10070
:101DF0002024002025732C25643A73557263517595
:101E0000657565207370696C6C6F766572A3A1004F
:101E100025732C25643A656332304174427566201F
:101E20007370696C6C6F7665722E2000BC01234262
:101E300025732C25643A636D645061636B20737065
:101E4000696C6C6F766572A3A1000000496E5061E9
:101E500072616D45727200004F7574506172616DF0
:101E60004572720052554E455252000052554E4F27
:101E70004B00000054494D454F555400CEB4D6AAEE
:101E8000B4EDCEF3000000002573202573000000A0
:101E900052445900454332302053746172742057C4
:101EA00061697465643A256420530000454332300B
:101EB00020C8EDB9D8BBFACAA7B0DCA3ACBCB4BD8E
:101EC000ABB6CFB5E7B9D8BBFAA3A1000FB42DE9E3
:101ED000F84F81460427F348C9EBC90100EB8104A0
:101EE000667E60680B90802000F0F2FF82460CABAB
:101EF0000093802150460B9A05F058FE8046B8F1B9
:101F0000000F02DDB8F1800F2FDD6522E6A1EEA003
:101F100001F076F802272BE0FFF760FD00251FFA9D
:101F200088F25146002001F01AFD14E0642003F00D
:101F3000BFF8E168EB4801F073FA206120690028DE
:101F400001DB032714E06169E64801F069FA002823
:101F500001DB02270CE028466D1C2189EDB2884286
:101F6000E4D34FF47A7003F0A3F8761EF6B2D3D21E
:101F7000504600F0E7FF00200090052F0ED2DFE86A
:101F800007F0030507090B00D7A408E0D9A406E071
:101F9000DBA404E0DCA402E0DDA400E0DEA448460B
:101FA00000F05AF901462246DEA000F0FDFF384657
:101FB000BDE8F80F5DF814FB02460021DBA3072003
:101FC00084E702460021082080E70246002109201C
:101FD0007CE72DE9F04104460F46224600210A2005
:101FE000FFF774FF0646032E20D1AE4D012C20D002
:101FF000022C25D0032C2AD0CEA1BA4801F010FA29
:10200000C5F82801D5F8280100280EDBD5F82811DD
:10201000B44830340830085CA04206D1D5F8281105
:10202000B0480A30085C312818D002263046BDE896
:10203000F081C0A1AB4801F0F3F9C5F82801E1E750
:10204000BFA1A84801F0ECF9C5F82801DAE7BFA163
:10205000A44801F0E5F9C5F82801D3E7D5F828111F
:10206000A04810230F3001442222384601F0FBF82B
:10207000DCE72DE9F04104252D2400210120FFF7A4
:1020800025FF984E874F09364FF4FA6815E0404611
:1020900003F00EF800210220FFF718FF0546032D7C
:1020A0000BD1B86C002807DDB86C805D312807D0F3
:1020B000B86C805D352803D00225641E601CE6D113
:1020C0002846B4E72DE9F04104251E240021032011
:1020D000FFF7FCFE834E734F0A364FF4FA6818E0A0
:1020E000404602F0E5FF00210420FFF7EFFE054621
:1020F000032D0ED1D7F88000002809DDD7F8800025
:10210000805D312808D0D7F88000805D352803D065
:102110000225641E601CE3D1284688E770B5054699
:102120001921284606F0AAF800210846FFF7CEFE3E
:102130000446032C09D15B4801696A481923083019
:1021400001440D22284601F08EF8204670BD10B5DE
:1021500000210520FFF7BAFE032801D07EA010BDA4
:10216000504C9C3420685F4908440D2105F0C3FFA2
:102170000021017021685B480A30084410BD70B529
:1021800005460020286000210620FFF79FFE044638
:10219000032C0AD14348D0F8B81052481923801DA7
:1021A00001442C22284601F05EF8204670BD2DE93E
:1021B000F04105460E466D480446FFF7AFFF032881
:1021C00009D06BA23146284605F016FD6BA000F041
:1021D00017FF02202BE7224619216CA000F0B6FE63
:1021E000FFF747FF0446032C09D06DA2314628466D
:1021F00005F002FD6DA000F003FF022017E7FFF7D6
:1022000061FFFFF7A4FF01466EA000F09FFE574854
:10221000001F0746FFF7B3FF3B466EA23146284634
:1022200005F0EAFC3A4603216DA000F08FFE20463F
:10223000FDE670B505460E462846FFF7BDFE28466A
:10224000FFF7BFFE0446032C03D131462846FFF7B3
:10225000C0FE204670BDB8E610B50B281DD2DFE8E1
:1022600000F006080A0C0E10121416181A0060A0CE
:1022700010BD62A010BD63A010BD64A010BD65A01C
:1022800010BD66A010BD69A010BD6BA010BD6DA0F3
:1022900010BD6FA010BD72A010BD75A000F0B0FE03
:1022A00079A010BD800200202E2E5C484152445778
:1022B0004152455C4C54455C454332305C65633269
:1022C000306E65742E63000025732C25643A636DAF
:1022D000645061636B207370696C6C6F766572A378
:1022E000A10000009A100020496E506172616D4596
:1022F000727200004F7574506172616D45727200A8
:1023000052554E455252000052554E4F4B00000060
:1023100054494D454F555400CEB4D6AAB4EDCEF332
:10232000000000002573202573000000434D494F35
:10233000540000002B51494143543A203100000021
:102340002B51494143543A20320000002B5149415E
:1023500043543A2033000000BBF1C8A1CDF8C2E7D6
:10236000D0C5CFA2CAA7B0DC210000008010002099
:10237000C7EBB2E5C8EB53494DBFA800CEB4BCECE7
:10238000B2E2B5BD53494DBFA800000053696DBF0F
:10239000A84943434944A3BA252E2A7300000000EC
:1023A00053494DBFA8C7B7B7D100000053494DC727
:1023B000B7B7D1CEDEB7A8D7A2B2E1C9CFCDF8C2A8
:1023C000E7000000CDF8C2E7D0C5CFA2A3BA2573BD
:1023D00000000000D0C5BAC5D6CAC1BF3A257300F7
:1023E0004C544520435351A3BA252E2A73000000B4
:1023F00051554552594943434944000053455443BC
:102400005300000051554552594353005345545011
:1024100053000000515545525950530051554552F3
:10242000594E4554494E464F000000005155455203
:102430005943535100000000434F46434F4E54450B
:1024400058540000414354434F4E544558540000E3
:102450004445414354434F4E5445585400000000F6
:102460005155455259434F4E5445585400000000B1
:102470004543323020CEDED0A7654E6574436D648F
:102480004E756D2100000000CEDEB4CBC3FCC1EE62
:102490000000000005280ED2DFE800F00305070960
:1024A0000B00D7A07047D9A07047DBA07047DCA015
:1024B0007047DDA07047DEA0704705280ED2DFE828
:1024C00000F0030507090B00DCA07047DEA0704791
:1024D000E0A07047E2A07047E4A07047E6A0704714
:1024E00070B5102000F0F4FC054629460120FFF7E6
:1024F00070FD032807D029460120FFF79AFE044605
:10250000032C02D005E0032070BD2946DDA000F0B9
:102510001DFD284600F016FD204670BD0FB42DE9C4
:10252000F84F81464FF00408DA48C9EBC90100EBC7
:102530008104667E60680B90802000F0C9FC8246B2
:102540000CAB0093802150460B9A05F02FFB0746F9
:10255000002F01DD802F2FDDCFA000F051FD4FF0C7
:1025600002082CE0FFF73AFA0025BAB251460020E3
:1025700001F0F5F916E0642002F09AFDE168D24816
:1025800000F04EFF20612069002802DB4FF00308B5
:1025900015E06169CC4800F043FF002802DB4FF0F2
:1025A00002080CE028466D1C2189EDB28842E2D376
:1025B0004FF47A7002F07CFD761EF6B2D2D250460D
:1025C00000F0C0FC4046FFF765FF04464846FFF7B1
:1025D00074FF01462246BDA000F0E6FC4046BDE87F
:1025E000F80F5DF814FB7CB5024600210220FFF7CE
:1025F00095FF0646032E2BD1002000900190162057
:1026000000F066FC0446A34DA96CAF480A30085C94
:102610002070A96CAC481023133001442C22601C9C
:1026200000F021FE601C05F0B1FDA96C1430A64A33
:102630000523114401442C22684600F014FE217841
:102640006B46621CA3A000F0AFFC204600F07AFCB1
:1026500030467CBD1CB50446CDE900230B46002165
:1026600022460846FFF75AFF03280ED189490B6915
:10267000954A303409329A5CA24205D10A699249DE
:102680000B31515C302900D002201CBD02460021D4
:10269000012043E770B504462078FFF7F7FF0328D1
:1026A0000CD1A38A628A2078611CFFF7D3FF05460C
:1026B000032D02D12078FFF796FF284670BD2DE943
:1026C000F84F06468A469146B9F1000F0DD0002515
:1026D000A84600240427FFF781F932786D4EB16DCA
:1026E0004B46002001F084F90DE00320BDE8F88F8F
:1026F000142002F0DDFC3E21734805F0FCFC10B113
:102700004FF0010804E028466D1CEDB24628EFD3D7
:10271000B8F1010F10D03846FFF7BCFE0446032085
:10272000FFF7CBFE01466848009077A3224679A0C8
:1027300000F066FC3846D9E74A465146002001F0D1
:102740000EF930E0642002F0B3FCF16F5E4800F057
:1027500067FEC6F88000D6F8800000280DDB03274E
:102760003846FFF797FE04460420FFF7A6FE014611
:10277000224656A000F018FCDCE7D6F88410524838
:1027800000F04EFE00280EDB02273846FFF782FEDF
:1027900004460420FFF791FE01464B4B224660A001
:1027A00000F02EFCC6E72046641CB6F87810A4B2F0
:1027B0008842C7D3BEE770B5054605245BA128460D
:1027C00000F02EFE002801DD002416E05CA1284662
:1027D00000F026FE002801DD04240EE05DA128465D
:1027E00000F01EFE002801DD022406E05EA128465E
:1027F00000F016FE002800DD0324204670BD000016
:10280000496E506172616D45727200004F7574506F
:102810006172616D4572720052554E455252000010
:1028200052554E4F4B00000054494D454F555400F2
:10283000CEB4D6AAB4EDCEF3000000004F50454E02
:10284000534F434B45540000434C4F5345534F4364
:102850004B4554005155455259534F434B45540035
:1028600054435053454E44434D4400005443505349
:10287000454E444255460000CEDEB4CBC3FCC1EE0B
:1028800000000000544350B1BEB5D84950A3BA254A
:1028900073000000B403002054637020636D645023
:1028A00061636B20D2E7B3F6A3A12D2DD4F6BCD380
:1028B0005443505F434D445041434B5F4C454ECAD7
:1028C000FDD6B5A1A30000009A1000202573202595
:1028D00073000000544350204368616E6E616CA326
:1028E000BA256320A1A320B7FECEF1C6F74950A3B5
:1028F000BA2573A1A320B7FECEF1C6F7B6CBBFDAD7
:10290000A3BA257300000000CEB4CAD5B5BD223EDF
:1029100022000000257320257320257320257300D5
:102920002573202573202573000000002B51495585
:1029300052433A2022636C6F7365642200000000EA
:102940002B51495552433A2022706470646561638B
:10295000742200002B51495552433A2022696E637C
:102960006F6D696E672200002B51495552433A2022
:1029700022696E636F6D696E672066756C6C2200EC
:102980000FB42DE9F84F81460427DF48C9EBC90190
:1029900000EB8104667E60680B90BD01284600F064
:1029A00097FA82465FEA0A0010D00CAB00932946E2
:1029B0000B9A05F0FBF88046B8F1000F01DDA84541
:1029C00038DDD2A000F01CFB022736E0DBA000F0CF
:1029D00017FB504600F0B6FA0220BDE8F80F5DF88C
:1029E00014FBFEF7FBFF00251FFA88F2514600207A
:1029F00000F0B5FF14E0642002F05AFBE168D7480C
:102A000000F00EFD20612069002801DB032714E09F
:102A10006169D24800F004FD002801DB02270CE0C8
:102A200028466D1C2189EDB28842E4D34FF47A70B8
:102A300002F03EFB761EF6B2D3D2504600F082FA88
:102A400000200090052F0ED2DFE807F003050709EC
:102A50000B00C3A408E0C5A406E0C7A404E0C8A412
:102A600002E0C9A400E0CAA4484600F020F90146EB
:102A7000BA4B2246C9A000F097FA3846ADE770B5C8
:102A80000446002122780846FFF77AFF032810D178
:102A900004F181031E46621C00210120FFF770FF34
:102AA00005463246611CC0A000F050FA032D01D04B
:102AB000284670BD04F20114002122780220FFF79D
:102AC0005FFF627800210320FFF75AFFA278002100
:102AD0000420FFF755FF284670BD70B5044610204E
:102AE00000F0F6F9054620782946FFF772FA032828
:102AF00007D020782946FFF79CFB0446032C02D020
:102B000005E0032070BD2946B1A000F01FFA284659
:102B100000F018FA204670BD2DE9F041B0F81431EC
:102B200000F5827200210520FFF72AFF03281CD13F
:102B30000A248A4E744D4FF4FA670D3612E0384677
:102B400002F0B6FA00210620FFF71AFF032809D188
:102B5000D5F8B810002904DDD5F8B810895D312901
:102B600003D00220641E611CE9D1BDE8F081002180
:102B70000E2005E770B500F58B7215460021072081
:102B8000FFF7FEFE032813D100210820FFF7F8FE0F
:102B90000446032C0BD15C48D0F8F000002805DD7A
:102BA00029466E4800F03CFC002800DC0224204648
:102BB00070BD10B50C46024600210920FFF7E0FE6B
:102BC000032801D0022010BD2146644800F028FCF3
:102BD000002801DD032010BD042010BD1CB500211C
:102BE0000091019102460A20FFF7CAFE032801D096
:102BF00000201CBD4448D0F82811584806230D3049
:102C000001440D22684600F02EFB684605F066FA86
:102C10001CBD0B46024600210D20B1E62DE9F84F00
:102C200083468A4617464FF0FF3844460025DFF8B2
:102C3000B091012089F80000FEF7DAFE324E0097CD
:102C4000D6F8381153465A46002000F0D1FE21E054
:102C5000642002F02DFA63A1644800F0E1FB00F16A
:102C60000904D6F84011614A3819104400F0D8FB25
:102C7000C6F84401D6F8440140B1D6F848115B4883
:102C800000F0CEFB002805DB44460AE0002C08DA01
:102C9000444606E028466D1CB6F83C11EDB2884269
:102CA000D6D3002089F800002046BDE8F88F0F2811
:102CB00027D2DFE800F0080A0C0E10121416181ABA
:102CC0001C1E202224004AA070474DA070474FA030
:102CD000704751A0704754A0704757A0704759A043
:102CE00070475CA070475FA0704762A0704765A006
:102CF000704767A0704769A070476CA070476EA0CE
:102D0000704770A0704700004004002046545020D7
:102D1000636D645061636B20D2E7B3F6A3A12D2DE0
:102D2000D4F6BCD34654505F434D445041434B5FAF
:102D30004C454ECAFDD6B5A1A30000004543323034
:102D400020467470436D645061636B20C4DAB4E64E
:102D5000B7D6C5E4CAA7B0DC210000009A10002055
:102D6000496E506172616D45727200004F7574500A
:102D70006172616D4572720052554E4552520000AB
:102D800052554E4F4B00000054494D454F5554008D
:102D9000CEB4D6AAB4EDCEF30000000025732025F2
:102DA000730D0A5B25735D00C5E4D6C3465450B766
:102DB000FECEF1C6F7557365726E616D653A257387
:102DC0002C2050617373776F72643A2573202E0044
:102DD000465450B1BEB5D84950A3BA25730000007F
:102DE000B4010020434F4E4E454354001A130020B7
:102DF000534554434F4E5445585449440000000035
:102E00005345544143434F554E5400005345544697
:102E1000494C4554595045005345545452414E5322
:102E20004D4F444500000000534554525354494D02
:102E3000454F5554000000004654504C4F47494EF2
:102E4000000000004745544C4F47494E53544154ED
:102E5000450000005345544449524543544F52598C
:102E6000000000004745544449524543544F5259CD
:102E7000000000004C49535446494C454E414D45D5
:102E80000000000047455446494C4553495A450007
:102E9000444F574E46494C450000000047455448B2
:102EA0004153444F574E53495A45000052454E41F5
:102EB0004D4546494C4500004654504C4F474F55F0
:102EC00054000000CEDEB4CBC3FCC1EE0000000015
:102ED00070B506463146002000F0AEFB04460020E7
:102EE00000F017FB05464B2D08D918225AA161A006
:102EF00004F076FE294663A004F072FE24B1314648
:102F0000204605F0BBF91BE0202253A159A004F094
:102F100067FE294663A004F063FE002000F0E0FA9B
:102F20003146002000F088FB04464CB925224AA116
:102F300050A004F055FE68A004F052FE04F068FCB6
:102F4000204670BD0146002000F06DBB0FB4F8B5FF
:102F500007AD00954FF480742046FFF7B9FF064691
:102F60005EA22146304604F047FE0446C4F5807157
:102F700030192B46069A04F019FE002806DD20447D
:102F800082B23146022000F0EAFC07E0502232A172
:102F900038A004F025FE50A004F022FE3046FFF7D2
:102FA000D1FFF8BC5DF814FB0FB4F8B507AD009580
:102FB0004FF480742046FFF78BFF064649A2214656
:102FC000304604F019FE0446C4F5807130192B46D2
:102FD000069A04F0EBFD002806DD204482B231465B
:102FE000022000F0BCFC07E06E221BA121A004F02F
:102FF000F7FD39A004F0F4FD3046FFF7A3FFD0E75A
:103000000FB4F8B507AD00954FF480742046FFF774
:103010005FFF064635A22146304604F0EDFD04462A
:10302000C4F5807130192B46069A04F0BFFD0028C4
:1030300006DD204482B23146022000F090FC07E019
:103040008B2205A10BA004F0CBFD23A004F0C8FD4A
:103050003046FFF777FFA4E72E2E5C5359535445B3
:103060004D5C535953504F52545C737973706F7267
:10307000742E63004C6F674572723A2025732C25BD
:10308000640000000D0AB6AFCCACC4DAB4E6D5BC1F
:10309000D3C3D2D1B3ACB9FDA3BA25642525A3A16E
:1030A0000D0A00000D0AC4DAB4E6D5BCD3C3A3BA36
:1030B000256425252D2DB6AFCCACC4DAB4E6D2E715
:1030C000B3F6A3A1B3F5CABCBBAFB6AFCCACC4DA00
:1030D000B4E6BFD5BCE4A3A1000000004C6F67417B
:1030E00070703A004C6F674465623A004C6F6745F8
:1030F00072723A0000210180418081804FF40061AA
:10310000801D05F0BBB82DE9F0418388161D3344BE
:103110004FF40067BB4202D30120BDE8F08145882F
:103120001223841D2B5543885B1CC3F30A03438081
:10313000458834232B5543885B1CC3F30A03438023
:1031400000230BE011F8015BB0F802C00CF804504A
:1031500045886D1CC5F30A0545805B1C9342F1DB75
:103160004288562111554188491CC1F30A0141800A
:103170004288782111554188491CC1F30A014180D8
:103180008188314481808188B94209D3FFF7B2FF39
:103190004322BFA1C5A004F023FDC8A004F020FD78
:1031A0000020BAE770B58388002B08D003889B1CE9
:1031B000C3F30A03038000231380831D21E0022050
:1031C00070BD1488641C14800488E45C01F8014B11
:1031D0000488641CC4F30A04048014888588AC4203
:1031E00003D20488B4F5006F0BD3FFF783FF662288
:1031F000A7A1AEA004F0F4FCB0A004F0F1FC022002
:1032000070BD0488E45C562CDBD10488641CC4F3D4
:103210000A040444A479782CD3D10188891CC1F311
:103220000A01018081881288891A091F8180002083
:1032300070BD2DE9F04105460C461746284604F0BE
:10324000A5FF0646384604F0A1FF3118A14204DB71
:1032500000212A19101A00F8011C39462846BDE839
:10326000F04104F0B2BF30B5054600205B1E04E01B
:103270002C54984204DA401C80B20C5C9442F7D182
:1032800030BD70B50446084611461D46049E04F044
:1032900032FF0246012006E0231803F8011CB04269
:1032A00004D8401C80B2115CA942F5D170BD30B584
:1032B00000231144491E18E00C7824090A2C01D27D
:1032C000302500E037252C4400F813400C7804F03A
:1032D0000F040A2C01D2302500E037252C4400EBE6
:1032E00043056C705B1C9BB2491E9342E4D330BD16
:1032F00030B500231AE0CD5C2C0905F00F05303401
:10330000392C03D9E41D00F8134001E000F8134004
:103310003035ECB2392C04D900EB4305E41D6C7058
:1033200002E000EB43056C705B1C9BB29342E2D35E
:1033300030BDF0B503460025084600260A2A01D014
:103340000670F0BD002B1DD005DA4FF02D0200F8FD
:10335000012BC3F1000342F210724FF00A0793FBF6
:10336000F2F454EA050C06D004F1300500F8015BD4
:1033700004FB1233012592FBF7F2002AEFDC067002
:103380000846F0BD3022027046700846F0BDF0B528
:1033900005460023002042F210720A26B5FBF2F423
:1033A000E4B254EA000704D030340746401CC0B2EF
:1033B000CC55B5FBF2F402FB1455B2FBF6F25B1CE4
:1033C000DBB2052BEAD308B9302008700846F0BDFF
:1033D0002DE9F04105460C46284604F0D7FE80B2A0
:1033E000002100B121700122002312E0AE5CEF5CED
:1033F000BE420CD1521C92B25B1C9BB2AE5CEF5C25
:10340000BE4201D0A35404E0E65CA65401E01BB127
:10341000E35C8242EAD380E6521C92B2A154F8E700
:103420002DE9F04782468946504604F0AFFE87B248
:10343000484604F0ABFE86B2002500243046FFF774
:1034400047FD804641464846FFF7C2FF0DE01AF8A7
:10345000050019F80410884204D16D1CADB2641C3B
:10346000A4B202E06CB118F80440BD4201D2B442EB
:10347000EDD34046FFF766FDB44205D3A81BBDE877
:10348000F0876D1CADB2F0E74FF0FF30F7E70000BA
:103490002E2E5C53595354454D5C5359534C49425D
:1034A0005C7379736C69622E630000004C6F674532
:1034B00072723A2025732C25640000000000000081
:1034C00003E011F8013B00F8013B521E531CF8D1F8
:1034D000704701E000F8011B521E531CFAD17047DF
:1034E00070B504466B486C4E002150F8240006EB82
:1034F000840542002869FFF7ECFF66480021103080
:1035000050F82420A868FFF7E4FF0120311908765D
:1035100070BD10B5002200215E4B5F4C53F8203087
:1035200004EB800005E0046934F8114004B1521C3A
:10353000491C8B42F7D864204243B2FBF3F0C0B27F
:1035400010BD2DE9F04105460F460024DFF8488103
:1035500008EB0500007E002803D1D8F800102846AB
:1035600088474FF0FF32FFB14A4E083656F8250023
:10357000B7FBF0F3B7FBF0F100FB117000B15B1C7F
:10358000444850F82510491E002921DB08EB850727
:10359000386930F811C0BCF1000F08D000249C42FB
:1035A00013D1002298B20AE01046BDE8F081641CF5
:1035B000F5E73C6901EB020C24F81C00521C9A420E
:1035C000F7D356F825004843EFE7491E0029E0DA13
:1035D0001046EAE770B5304A13181B7E002B13D053
:1035E0002C4B103353F820308B421AD9294B083317
:1035F00053F82030B1FBF3F102EB8002106930F890
:1036000011300020002408E011688847012070BDB7
:1036100015690E1825F81640401C9842F8DB00206A
:1036200070BD022070BD002905D01B4A02EB80024C
:103630009268891ACEE7704710B504462046FFF716
:1036400080FF411C05D0144901EB840189680844BE
:1036500010BD002010BD2DE9F041064688461746F2
:1036600039463046FFF76DFF0446601C0FD00A480C
:103670003A4600EB86054146A8682044FFF720FF44
:1036800041463046FFF7CFFFA86820448DE7002071
:103690008BE70000B4BE0008E405002010B50C461E
:1036A000F24A52F82030002B09D05222F0A1F6A0A5
:1036B00004F096FAF8A004F093FA204610BD42F800
:1036C0002040FAE730B40C46E84951F82030002B8E
:1036D00003D0204630BC1146184730BC70477047B5
:1036E0007047F449C2B28B689A8089680A8852068A
:1036F000FCD570472DE9F04387B004460D461646C9
:1037000098460121084602F01AFBEA4818220F38B1
:10371000015D401F005D00F011FFE6480422401FDC
:10372000015D401F005D00F009FFE348002C7CD0E4
:1037300050F82400012102F00DFB02950025ADF8A0
:103740000C50ADF80E50ADF81050ADF81450ADF867
:103750001260D84E02A956F8240002F08FFB56F8EA
:1037600024004FF4587102F0D9FCBDF8120006F1A4
:103770001409000722D5042C20D056F82400012279
:10378000802102F01DFCCC4F00950195183F59F89F
:103790002410385D1023002200F027FC06F12400DD
:1037A000002150F82420385D00F01CFBAF480121B7
:1037B000303850F82420385D00F014FBBDF81200BA
:1037C000400759D5BC481038005D8DF818008DF8B9
:1037D00019808DF81A5001208DF81B0006A801F001
:1037E000E8FF56F82400012240F2244102F0CDFB0C
:1037F000042C3BD056F824000122402102F0E0FBCB
:10380000CDE90058AC4859F824101430A0F128052F
:1038100050F82420285D002300F0E7FB05F10A00A2
:10382000A64F30F81410285D00E01AE057F8200089
:1038300003F07EFF8D480021203850F82420285DB9
:1038400000F0D0FA89480121103850F82420285D72
:1038500000F0C8FA285D012157F8200003F051FF5D
:103860000AE00068012102F06AFA66E7012240F2EC
:103870002551306902F089FB56F82400012102F03D
:1038800078FB07B0BDE8F0831CB5044689480122E7
:10389000802150F8240002F093FB06200021CDE99E
:1038A0000010844810231430002250F8241082485D
:1038B0001838005D00F099FB1CBD7CB504467D48BE
:1038C0000122402150F8240002F07AFB062000215A
:1038D000CDE900107848784D1430143D50F824207C
:1038E00074480023143050F82410285D00F07DFB4C
:1038F00005F10A00714E30F81410285D56F82000CA
:1039000003F016FF285D012156F82000BDE87C4039
:1039100003F0F7BE2DE9F0410446674D674E143DB4
:103920000021285D56F8200003F0EBFE05F10A07A0
:1039300005F1280037F8141050F8240004F09EFC1C
:10394000285D37F8141056F8200003F0F1FE285DCA
:10395000012156F82000BDE8F04103F0D2BE2DE968
:10396000F047044688461646B8F1000F25D0002ED1
:1039700023D0042C23D0504FDFF84091183F002172
:10398000385D59F8200003F0BCFE4A4D0020183D78
:103990002855385D59F82000C0F80C80385D314654
:1039A00059F8200003F0C4FE385D012159F82000C9
:1039B00003F0A7FE285D0028FCD0BDE8F0870025B5
:1039C0003C4F4021386902F0A2FB0EE018F80510C8
:1039D00057F8240002F02EFB57F82400402102F093
:1039E00096FB0028F8D06D1CADB2B542EED3E4E7EB
:1039F0000FB470B586B004460CA801902D4E10E0AF
:103A00005C2916D025295BD0401C0B9056F8240069
:103A100002F010FB56F82400402102F078FB002849
:103A2000F8D00B9801780029EAD106B070BC5DF897
:103A300014FB401C0B9001786E290DD0722902D026
:103A4000401C0B90E6E756F824000D2102F0F2FA34
:103A50000B98401C0B90DDE756F824000A2102F079
:103A6000E9FA0B98401C0B90D4E70000305B002073
:103A70002E2E5C53595354454D5C55534152545C62
:103A800075736172742E63004C6F674572723A20D1
:103A900025732C2564000000556172742043616C0D
:103AA0006C6261636B20726570656174207265671A
:103AB000210000001C060020E4BE0008540600207F
:103AC000401C0B90017864291BD0732902D0401C44
:103AD0000B909FE7019820C801900BE056F8240056
:103AE00002F0A8FA56F82400402102F010FB00284A
:103AF000F8D06D1C29780029F0D10B98401C0B9050
:103B000088E7019808C801900A2202A91846FFF721
:103B100010FC02AD0BE056F8240002F08BFA56F8C8
:103B20002400402102F0F3FA0028F8D06D1C297817
:103B30000029F0D10B98401C0B906BE770B59D4CA1
:103B400040F22441204602F0EDFAA0B19A4D002146
:103B5000286903F0D6FD2088201D0088286903F01D
:103B6000E9FDC0F5807082B294490020FFF7AAFDFC
:103B70000020FFF7CFFE40F225552946204602F0EF
:103B8000D1FA18B12946204602F0ECFA40F2277526
:103B90002946204602F0C6FA002806D029462046CB
:103BA000BDE87040002202F0F0B970BD70B5844CE1
:103BB00040F22441204602F0B5FAA0B17E4D00212A
:103BC000686903F09EFD2088201D0088686903F065
:103BD000B1FDC0F5807082B27A490120FFF772FD15
:103BE0000120FFF797FE40F225552946204602F0B6
:103BF00099FA18B12946204602F0B4FA40F2277526
:103C00002946204602F08EFA002806D02946204692
:103C1000BDE87040002202F0B8B970BD70B56A4CC2
:103C200040F22441204602F07DFAA0B1624D00210D
:103C3000A86803F066FD2088201D0088A86803F0AE
:103C400079FDC0F5406082B260490220FFF73AFD7D
:103C50000220FFF75FFE40F225552946204602F07C
:103C600061FA18B12946204602F07CFA40F2277525
:103C70002946204602F056FA002806D0294620465A
:103C8000BDE87040002202F080B970BD70B5504CA4
:103C900040F22441204602F045FAA0B1464D0021F1
:103CA000686A03F02EFD2088201D0088686A03F0F2
:103CB00041FDC0F5807082B246490320FFF702FD46
:103CC0000320FFF727FE40F225552946204602F043
:103CD00029FA18B12946204602F044FA40F2277525
:103CE0002946204602F01EFA20B10022294620462D
:103CF00002F04BF92046BDE87040402102F00EBAB8
:103D00002DE9F041344D40F22551284602F00AFADF
:103D1000324C002658B1AA882168481C20603048DF
:103D20004254216846542068FF2800DB266040F298
:103D300024473946284602F0F5F988B12888A88832
:103D40002068274982B20420FFF7BCFC4FF4807141
:103D5000234804F0B5FA26603946284602F002FAF4
:103D600040F227742146284602F0DCF9002806D0EC
:103D700021462846BDE8F041002202F006B9BDE820
:103D8000F08116490120091D087070471349012070
:103D9000091D4870704711490120091D887070473E
:103DA0000E490120091DC870704770477047704761
:103DB000704700000038014054060020445B00209A
:103DC00000440040445C002000480040445D002066
:103DD000004C0040446900200050004000060020D4
:103DE000446A002010B5144600290BD0012919D0CF
:103DF0004E22F1A1F5A003F0F3FEF8A003F0F0FECF
:103E0000204610BDFE4951F8202042B14322EAA1CC
:103E1000EEA003F0E5FEFBA003F0E2FEF0E741F8C0
:103E20002040EDE7F649303151F8202042B14A22D6
:103E3000E1A1E6A003F0D4FEF9A003F0D1FEDFE794
:103E400041F82040DCE730B4ED49B0F1007F01F1EA
:103E500030026FD036DCB0F5005F6CD018DC802803
:103E600079D00ADC02286AD008286DD0202870D1C9
:103E7000486800286DD030BC0047B0F5007F6FD097
:103E8000B0F5006F65D19068002862D030BC004763
:103E9000B0F5002F74D00ADCB0F5004F6AD0B0F551
:103EA000003F56D10869002853D030BC0047B0F518
:103EB000001F6AD0B0F5000F4BD15069002848D0E0
:103EC00030BC0047DD4C031BA04278D018DCDC4C32
:103ED000A0EB0403A04267D009DCB0F1006F5ED014
:103EE000981D36D1C86900287DD030BC0047182BFA
:103EF00060D0782B77D1106A002874D030BC00478E
:103F0000B3F5FC4F65D00ADCB3F5C06F5CD0B3F5F8
:103F1000F05F68D1886A002865D030BC0047B3F5EF
:103F2000FF3F5BD0C748C3425DD1D06A00285AD05A
:103F300030BC00472EE018E00DE000E004E0086827
:103F4000002850D030BC0047106800284BD030BC4F
:103F5000004748E004E05068002844D030BC0047E7
:103F6000886800283FD030BC0047C86800283AD095
:103F700030BC0047D068002835D030BC0047FFE790
:103F8000106900282FD030BC0047486900282AD08B
:103F900030BC00478869002825D030BC00479069B4
:103FA000002820D030BC0047D06900281BD030BC8E
:103FB000004704E0086A002815D030BC0047486A72
:103FC000002810D030BC0047506A00280BD030BC0D
:103FD0000047906A002806D030BC0047C86A002815
:103FE00001D030BC004730BC70472DE9F0478CB0A1
:103FF0000446DDE914980D4617469A46072C04D26C
:104000000121084601F090FE03E00121022001F0A9
:104010008BFE8D4E56F8240003F0D2FA01950297DC
:10402000CDF80CA0002504950595802006900795F5
:104030000895CDF8249040010A900B9556F824007D
:1040400001A903F034FB814810F824008DF800002A
:104050008DF801808DF8025001208DF8030068462C
:1040600001F0A7FB56F824000122022103F056FBC1
:104070000CB0BDE8F08710B5022003F05EFB01280C
:1040800005D1022003F081FB0220FFF7DCFE0820AF
:1040900003F053FB01280ED1082003F076FBD52254
:1040A00045A14AA003F09CFD69A003F099FDBDE87D
:1040B00010400820C7E610BD10B5202003F03DFBDE
:1040C000012805D1202003F060FB2020FFF7BBFE74
:1040D000802003F032FB01280ED1802003F055FB35
:1040E000EB2235A139A003F07BFD5CA003F078FD45
:1040F000BDE810408020A6E610BD10B54FF4007456
:10410000204603F01AFB012805D1204603F03DFBB1
:104110002046FFF798FE4FF40064204603F00DFBA5
:1041200001280FD1204603F030FB40F2011222A1FA
:1041300026A003F055FD4CA003F052FD2046BDE83B
:10414000104080E610BD10B54FF40054204603F037
:10415000F4FA012805D1204603F017FB2046FFF7AB
:1041600072FE4FF40044204603F0E7FA01280FD115
:10417000204603F00AFB40F217120FA113A003F030
:104180002FFD3CA003F02CFD2046BDE810405AE670
:1041900010BD10B54FF40034204603F0CEFA0128CC
:1041A00005D1204603F0F1FA2046FFF74CFE4FF40C
:1041B0000024204664E000002E2E5C5359535445E1
:1041C0004D5C444D415C646D612E63004C6F6745EE
:1041D00072723A2025732C2564000000446D6154EE
:1041E000652043616C6C6261636B2022654972716A
:1041F0005479706522206572726F72210000000090
:10420000446B0020446D6154632043616C6C6261B7
:10421000636B2072657065617420726567210000B0
:10422000446D6154652043616C6C6261636B207204
:1042300065706561742072656721000000020010DE
:10424000080000100002F8FF5406002008BF000814
:10425000444D41315F54453121000000444D41310E
:104260005F54453221000000444D41315F544533D5
:1042700021000000444D41315F54453421000000CD
:1042800003F05BFA012811D1204603F07EFA40F2D8
:104290002D12AFF2DC01AFF2CC0003F0A1FC8BA039
:1042A00003F09EFC2046BDE81040CCE510BD10B5E3
:1042B0004FF40014204603F040FA012805D12046AF
:1042C00003F063FA2046FFF7BEFD4FF400042046DA
:1042D00003F033FA012811D1204603F056FA40F2D8
:1042E0004312AFF22C11AFF21C1003F079FC7AA04C
:1042F00003F076FC2046BDE81040A4E510BD10B5E3
:104300004FF00074204603F018FA012805D120462A
:1043100003F03BFA2046FFF796FD4FF0006420467D
:1043200003F00BFA012811D1204603F02EFA40F2D7
:104330005912AFF27C11AFF26C1003F051FC69A07E
:1043400003F04EFC2046BDE810407CE510BD10B5E2
:10435000674C204603F0F1F9012805D1204603F00F
:1043600014FA2046FFF76FFD614CA41D204603F0B0
:10437000E4F9012811D1204603F007FA40F26F1248
:10438000AFF2CC11AFF2BC1003F02AFC59A003F03D
:1043900027FC2046BDE8104055E510BD10B5544C33
:1043A0001E34204603F0C9F9012805D1204603F048
:1043B000ECF92046FFF747FD4D4C7E34204603F0D4
:1043C000BCF9012811D1204603F0DFF940F2851233
:1043D000AFF21C21AFF20C2003F002FC45A003F069
:1043E000FFFB2046BDE810402DE510BD10B5444C44
:1043F000204603F0A2F9012805D1204603F0C5F9B3
:104400002046FFF720FD3F4C204603F096F9012897
:1044100011D1204603F0B9F940F29B12AFF26821A6
:10442000AFF2582003F0DCFB37A003F0D9FB2046A5
:10443000BDE8104007E510BD10B5364C204603F02E
:104440007CF9012805D1204603F09FF92046FFF7AB
:10445000FAFC314C204603F070F9012810D12046B7
:1044600003F093F940F2B112AFF2B421AFF2A420FD
:1044700003F0B6FB29A003F0B3FB2046FFF7E3FCF3
:10448000294C204603F059F9012805D1204603F0B4
:104490007CF92046FFF7D7FC244C204603F04DF969
:1044A000012811D1204603F070F94FF4DF72AFF20A
:1044B000F821AFF2E82003F093FB1DA003F090FB7E
:1044C0002046BDE81040BEE410BD0000444D41311F
:1044D0005F54453521000000444D41315F5445365D
:1044E00021000000444D41315F5445372100000058
:1044F00002000010444D41325F544532210000005B
:104500000002001000080010444D41325F54453352
:10451000210000000020001000800010444D4132B6
:104520005F54453421000000000002100000081014
:10453000444D41325F54453521000000F8B5044632
:104540000D4616469848012150F8240001F0F7FB6B
:1045500095481C3030F81500ADF800008DF8036068
:1045600003208DF802009148694650F8240001F0BC
:10457000E0F9F8BD2DE9FE430646DDF828900C462B
:10458000154698462A4621463046FFF7D7FF282D84
:1045900001D0482D36D10121084601F0D0FB824FD1
:1045A0008C37385D8DF800008DF8019000258DF86E
:1045B00002508DF80350684601F0FBF8A7F1500057
:1045C000015D4438805D01F070FAA7F1400656F8AD
:1045D000240001908DF808508DF8098001258DF890
:1045E0000A5001A801F04AFE56F8240001F0A5FE89
:1045F000385700F01F018D404009800000F1E02095
:10460000C0F80051BDE8FE83684A52F82000C26835
:10461000654B1C3333F811104A40C260704710B527
:104620000C46634A52F82030002B09D0952261A134
:1046300065A003F0D5FA68A003F0D2FA204610BDB9
:1046400042F82040FAE770B5064600204FF080415E
:1046500005F0B6F904460D46304605F04FFE05F06C
:10466000AFF922462B4605F041FC05F0D3FD504939
:1046700051F82000002802D0BDE87040004770BD0E
:1046800010B5012001F03EFE28B1012001F043FEEB
:104690000120FFF7D8FFBDE81040012001F04DBE1A
:1046A00010B5022001F02EFE012805D1022001F0F4
:1046B00032FE0220FFF7C7FFBDE81040022001F0E4
:1046C0003CBE10B5042001F01DFE28B1042001F00D
:1046D00022FE0420FFF7B7FFBDE81040042001F0E0
:1046E0002CBE10B5082001F00DFE012805D10820D0
:1046F00001F011FE0820FFF7A6FFBDE810400820DA
:1047000001F01BBE10B5102001F0FCFD28B11020F7
:1047100001F001FE1020FFF796FFBDE810401020C9
:1047200001F00BBE30B591B005241F4D4C3555F846
:10473000240001F0F4FD88B155F8240001F0EBFDF0
:10474000402101A803F0BCFD234629A2402101A875
:1047500003F052FA55F82400FFF775FF641C092C8A
:10476000E5DD11B030BD30B591B00A240E4D4C35A9
:1047700055F8240001F0D3FD88B155F8240001F06C
:10478000CAFD402101A803F09BFD234618A2402149
:1047900001A803F031FA55F82400FFF754FF641C18
:1047A0000F2CE5DDDDE7000040BF00088406002097
:1047B000A46B00202E2E5C53595354454D5C494F39
:1047C0005C696F2E630000004C6F674572723A207F
:1047D00025732C2564000000494F2043616C6C62F6
:1047E00061636B207265706561742072656721007A
:1047F0004558544925642049525121000021016047
:104800004160018181720B2210A103F080BD0EB5C1
:10481000114A12680092104A121D126801920E4A43
:1048200008321268029200290BD0012904D00C2210
:104830006946FEF75DFD0EBD0C226946FEF758FD88
:104840000EBD0C22694603F062FD0EBD4465632077
:104850003137203230323300E8F7FF1F10B50C46F5
:10486000F54901280BD0022816D03D22F3A1F8A06B
:1048700003F0B6F9FAA003F0B3F9204610BD48687A
:1048800040B13222EDA1F2A003F0AAF9FBA003F09F
:10489000A7F9F2E74C60F0E7886840B13922E7A158
:1048A000EBA003F09DF9FDA003F09AF9E5E78C6019
:1048B000E3E7E149012805D0022807D188680028EC
:1048C00004D000474868002800D00047704710B562
:1048D000012001F0F2FD38B1012001F0FCFD01F0F2
:1048E000CDFD0120FFF7E5FF022001F0E6FD0028E5
:1048F00008D0022001F0EFFD01F0C0FDBDE810403E
:104900000220D6E710BD10B5022001F0D6FD002828
:104910000CD04FF4003001F010FD022001F0DBFD5F
:1049200001F0ACFDBDE810400220C2E710BD30B57B
:104930006423B0FBF3F4E4B2B0FBF3F503FB150022
:10494000132C01D96430C0B200EB90030724B3FBF1
:10495000F4F504FB1533D94D1A440D4415F8015CE8
:104960002A4492B2800703D1032901D2521E92B287
:10497000B2FBF4F004FB102030BD810701D0002011
:1049800070476421B0FBF1F201FB120109B1012073
:1049900070474FF4C871B0FBF1F201FB120008B18F
:1049A00000207047012070472DE9F04788B0044689
:1049B00001F06AFD01F039FD0646DFF80483B6FB1D
:1049C000F8F39D480A270188994279D0038040F284
:1049D000B2754FF4B7794FF4B67A0FE02846FFF777
:1049E000CCFF38B14B4502D3A3F5B77304E06D1C7F
:1049F000ADB205E0A3F26D136D1CADB25345EDD819
:104A00000195BDF804104FF47A70B1FBF0F130312C
:104A10002170BDF80410B1FBF0F200FB121264210A
:104A2000B2FBF1F230326270BDF80420B2FBF0F557
:104A300000FB1520B0FBF1F201FB1200B0FBF7F018
:104A40003030A070BDF80400B0FBF7F107FB110097
:104A50003030E0700025DFF8649209F10C090DE0B8
:104A6000BDF80400FFF789FF08B1012D7AD019F8CD
:104A70000500984204D81B1A6D1CADB21C2BEFD256
:104A80006D1C04955B1C03939DF81000B0FBF7F0C0
:104A9000303060719DF81000B0FBF7F107FB11009A
:104AA0003030A0719DF80C00B0FBF7F03030207270
:104AB0009DF80C00B0FBF7F107FB1100303060727D
:104AC000B6FBF8F008FB10604FF46161B0FBF1F247
:104AD0000792B0FBF1F201FB12033C22B3FBF2F3AD
:104AE0000693B0FBF1F301FB1300B0FBF2F102FB04
:104AF000110005909DF81C00B0FBF7F03030E0721B
:104B00009DF81C00B0FBF7F107FB1100303020735B
:104B10009DF81800B0FBF7F03030A0739DF8180036
:104B2000B0FBF7F107FB11003030E0739DF8140083
:104B3000B0FBF7F0303060749DF81400B0FBF7F173
:104B400007FB11003030A0749DF80C209DF8101068
:104B5000BDF80400FFF7EBFE029008B00320BDE8AB
:104B6000F087FFE71D2B8BD31D3B85E755481BE7DF
:104B700008B503218DF800108DF8010000208DF894
:104B8000020001208DF80300684600F012FE08BD07
:104B90002DE9F041074600244A48202181722D2149
:104BA000C17101713A210174417301214FF0C0506C
:104BB00001F0D0F80121084601F0C1F8012001F010
:104BC000D1FB042001F028FB45F25006B04232D060
:104BD00001F0F8FA012001F03CF801F018FC01F0B6
:104BE0004DFC6FF07F4500E0641C412000F0B6FFF3
:104BF00008B9AC42F8D3DFF8D080444505D24FF471
:104C0000807001F03BF8012466E00024012001F0EF
:104C100032F800E0641C612000F0A0FF08B9AC424B
:104C2000F8D3444570D24FF4007001F027F8CA223F
:104C300002A107A04AE079E0A00600202E2E5C53D6
:104C4000595354454D5C5254435C7274632E630057
:104C50004C6F674572723A2025732C256400000062
:104C60005274635F526567486F6F6B43616C6C622F
:104C700061636B204661696C656421005274632036
:104C800053656354692043616C6C6261636B20728D
:104C9000657065617420726567210000527463203D
:104CA000416C7254692043616C6C6261636B207269
:104CB000657065617420726567210000DCBF0008C3
:104CC00080510100E46B0020F0FFFF0002F088FF3C
:104CD000C9A002F085FF0024012000F0D4FF01F0FC
:104CE000CDFBF4B147F6FF7001F0AFFB01F0C6FB5E
:104CF00001F0C4FB01F092FB01F0C0FB314604203F
:104D000001F082FA18E0FFE7CF22AFF2D001AFF254
:104D1000C00002F065FFB8A002F062FF0220BDE80B
:104D2000F08149F6404001F090FBDFE701F0A6FB7F
:104D30000121084601F060FB01F0A0FB01210846BB
:104D400001F05AFB01F09AFB0121022001F054FB13
:104D500001F094FB002001F005FB3846FFF708FF47
:104D6000A648FFF721FEAFF2FB110120FFF776FD09
:104D70000320D4E72DE9F05F00230178C2783039B1
:104D800001EB4104C4EBC11102EBC1044278642180
:104D9000303A4A438178303901EB810102EB41011D
:104DA000214430398DB241798279303901EB810467
:104DB0006FF02F0101EB44042244D7B2027A447A07
:104DC000303A02EB820201EB42022244D6B2C27AAE
:104DD000047B303A02EB820201EB4202224402F0F1
:104DE000FF08827BC47B303A02EB820201EB420275
:104DF000224402F0FF09827C407C303800EB8000C6
:104E000001EB4000104400F0FF0AA5F2B2708228C6
:104E100002D30220BDE8F09F40F2B274DFF8E0B1A7
:104E200009E02046FFF7A9FD08B15B4401E07548A1
:104E30000344641CA4B2AC42F3D37F1EFFB200242F
:104E4000DFF8C4B110E01BF8040040F2A32148438E
:104E500003EBC0132846FFF790FD18B1012C01D1D8
:104E60006A480344641CA4B2BC42ECD3761E40F2F0
:104E7000A320464303EBC610C8EB4811C1EB082141
:104E800000EB0110C9EB091100EB810000EB0A04F3
:104E9000012001F067FA01F0BAFA01F0EFFA2046BA
:104EA00001F0CCFA01F0EAFA01F0B8FA01F0E6FA02
:104EB0000320AFE72DE9F05F00230178C278303995
:104EC00001EB4104C4EBC11102EBC104427864213F
:104ED000303A4A438178303901EB810102EB4101DC
:104EE000214430398DB241798279303901EB810426
:104EF0006FF02F0101EB44042244D7B2027A447AC6
:104F0000303A02EB820201EB42022244D6B2C27A6C
:104F1000047B303A02EB820201EB4202224402F0AF
:104F2000FF08827BC47B303A02EB820201EB420233
:104F3000224402F0FF09827C407C303800EB800084
:104F400001EB4000104400F0FF0AA5F2B270822885
:104F500001D302205EE740F2B274DFF8A4B009E0AA
:104F60002046FFF70AFD08B15B4401E025480344F1
:104F7000641CA4B2AC42F3D37F1EFFB20024DFF85E
:104F800088B010E01BF8040040F2A321484303EB73
:104F9000C0132846FFF7F1FC18B1012C01D11B48C2
:104FA0000344641CA4B2BC42ECD3761E40F2A3209E
:104FB000464303EBC610C8EB4811C1EB082100EBD8
:104FC0000110C9EB091100EB810000EB0A0401207C
:104FD00001F0C8F901F01BFA01F050FA204601F087
:104FE0003CFA01F04BFA01F019FA01F047FA0020FF
:104FF00001F0B8F903200DE700000000E46B002089
:105000000085E2018033E101E8BF00088051010022
:10501000354840683221B0FBF1F201FB1200002854
:1050200001D1FCF792B8704710B5042000F004FCE1
:105030002E482F492C4A0068B0FBF1F31370B0FBE7
:10504000F1F142F2107041430A2050804FF0E0200D
:10505000026942F0020202614161016941F001010D
:10506000016110BD70B505462248854208D9054644
:10507000502221A127A002F0B3FD2AA002F0B0FD2A
:1050800000214FF0E0267469174800784543B36962
:10509000B2699A42FCD003D2A3EB0200014403E0C0
:1050A000A4EB0200184401441346A942F0D370BD9A
:1050B00070B5054600244FF47A7605E03046FFF7D8
:1050C000D1FF00F06FF9641CAC42F7D370BD70B52E
:1050D000054600244FF47A7603E03046FFF7C2FF1E
:1050E000641CAC42F9D370BDAC060020E006002081
:1050F00040420F00E3388E032E2E5C535953544523
:105100004D5C5359535449434B5C737973746963D1
:105110006B2E63004C6F674572723A2025732C2505
:10512000640000000000000010B50C467E4A52F8F2
:105130002030002B09D034227CA182A002F050FD47
:1051400084A002F04DFD204610BD42F82040FAE751
:10515000754951F82000002800D0004770472DE91C
:10516000FF410446884615461F4641F69910804582
:1051700008D980465E226DA172A002F031FD75A0B3
:1051800002F02EFD7448012150F8240000F0E2FDE9
:10519000714E083E305D8DF80C008DF80D500025E5
:1051A0008DF80E508DF80F5003A800F002FB41F669
:1051B0001F40ADF80000ADF80650ADF80250404673
:1051C00005F09CF8654A664B04F090FE0022654BA2
:1051D00005F0B2F905F04EF8ADF804008DF808506E
:1051E000614D694655F8240001F066FA012255F830
:1051F0002400114601F04BFD55F82400394601F01A
:105200002CFD55F82400012101F080FF30570121C9
:1052100000F01F0291404009800000F1E020C0F83A
:105220000011BDE8FF81504951F82000002101F034
:1052300035BF70B504464C4D002155F8240001F0EF
:105240002DFF55F82400BDE87040012101F005BD97
:10525000454951F82000002101F0FFBC10B50121A3
:105260008C07204601F046FF012807D10121204686
:1052700001F04CFFBDE81040002069E710BD10B5FB
:105280003A4C0121204601F035FF012807D10121C8
:10529000204601F03BFFBDE81040012058E710BD5B
:1052A00010B5334C0121204601F024FF012807D11D
:1052B0000121204601F02AFFBDE81040022047E707
:1052C00010BD10B52B4C0121204601F013FF012821
:1052D00007D10121204601F019FFBDE8104003204D
:1052E00036E710BD10B5244C0121204601F002FF25
:1052F000012807D10121204601F008FFBDE8104038
:10530000042025E710BD10B51C4C0121204601F0FA
:10531000F1FE012807D10121204601F0F7FEBDE88A
:105320001040052014E710BDF86B00202E2E5C53B2
:10533000595354454D5C54494D45525C74696D65F3
:10534000722E63004C6F674572723A2025732C25CC
:105350006400000000000000FCBF00089A999999C1
:105360009999B93F0000F03FB406002000040040C6
:1053700000080040000C00400010004000140040F5
:1053800010B545F2555000F0FFFE062000F0FFFE7C
:1053900040F20D3000F0FEFE00F0FFFEBDE81040D0
:1053A00000F000BF00F0F9BE03E010F8013B01F887
:1053B000013B521E92B2F8D270472DE9F0410546EA
:1053C0000E461746002407E0284601F0C3FF26F8E2
:1053D0001400AD1C641CA4B2BC42F5D3BDE8F0813E
:1053E0002DE9F0410E4617460546002409E036F83F
:1053F0001410284601F0B0FF0428EFD1AD1C641C46
:10540000A4B2BC42F3D3E9E72DE9F04FADF6040DA9
:1054100082460F461546AAF10064B4F1005F04D33A
:1054200000200DF6040DBDE8F08F212000F096FB62
:10543000012809D06B22A3A1A8A002F0D1FBABA048
:1054400002F0CEFB0220ECE701F07DFE4FEAD4280B
:10545000C4F34906C6F58064A54200D82C460DF178
:10546000040B37E032183BF812208A4203D1401C6B
:1054700080B2A042F6D3A04214D2484601F09CFE6E
:10548000002006E0821937F810102BF81210401C8B
:1054900080B2A042F6D348464FF4806201A9FFF7DC
:1054A0009FFF04E0224639465046FFF799FFA54288
:1054B00003D101F054FE0320B3E708F101080026F0
:1054C00007EB4407A244281B85B24FF48064A54231
:1054D00000D82C464FF0006000EBC829421401A907
:1054E0004846FFF76AFF00204FF6FF71C1E72DE93C
:1054F000F04107460E46002402F0010000EB520581
:10550000212000F02BFB012809D0A8226DA173A057
:1055100002F066FB75A002F063FB02205EE701F07B
:1055200012FEA7F10060B0F5002F01D278050BD074
:10553000AE2264A169A002F053FB6CA002F050FB04
:1055400001F00DFE022049E7B5F5006F0BD9B4223A
:105550005CA162A002F044FB64A002F041FB01F0F8
:10556000FEFD02203AE7352002F011F8384601F03E
:1055700023FE04281BD0BB2252A158A002F030FB0E
:105580005AA002F02DFB12E00A20FFF791FD0A2C31
:105590000BD9C2224BA151A002F022FB53A002F072
:1055A0001FFB01F0D0FD022018E7641CA4B201200B
:1055B00001F0DEFF0128E7D023E0202001F0E7FF23
:1055C00030787178B61C40EA0121384601F0C4FEFB
:1055D000002410E00A20FFF76BFD1E2C09D9D3220E
:1055E00038A13EA002F0FCFA40A002F0F9FA022035
:1055F000F4E6641CA4B2202001F0BAFF0128E9D12E
:10560000BF1C6D1EADB2D8D201F0A9FD0320E5E6A6
:105610002DE9F0478146884600260024002702F045
:10562000010000EB5205212000F098FA01280AD071
:10563000F12224A129A002F0D3FA2CA002F0D0FA82
:105640000220BDE8F08701F07EFD352001F09FFFCC
:1056500012E00A20FFF72CFD0A2C0BD9FB2219A11E
:105660001EA002F0BDFA21A002F0BAFA01F06BFD13
:105670000220E6E7641CA4B2012001F079FF0128B2
:10568000E7D018E0202001F082FF701C18F8061007
:1056900080B2421C18F8000096B241EA002A09EBD9
:1056A0000704600502D1204601F086FD20465146E0
:1056B00001F052FEBF1C6D1EADB2E3D201F04FFDF2
:1056C0000320BEE72E2E5C53595354454D5C464C87
:1056D0004153485C666C6173682E63004C6F67458C
:1056E00072723A2025732C2564000000000000002F
:1056F000FEB505460E460121084600F020FB4FF49A
:105700008037019700248DF808408DF80950012555
:105710008DF80A5001A800F0B1FD384600F00DFEEA
:105720008DF800508DF801608DF802408DF803402F
:10573000684600F03EF81B4902200860C02000F0D7
:1057400017FE012000F011FEFEBD3EB50121080745
:1057500000F000FB01248DF808408DF80940002579
:105760008DF80A508DF80B4002A800F022F8684628
:1057700000F0BBFD200400908DF8045008208DF847
:1057800005008DF80640684600F078FDC02000F066
:10579000EFFD012000F0E9FD3EBD4FF4803000F048
:1057A000CCBD000000E100E02A4908432A49086016
:1057B000704770B50F23C27801260178002A1ED0E9
:1057C000254A126802F4E062C2F5E062120AC2F1F0
:1057D0000404D3404578A54082781A402A43120138
:1057E00001F1E02181F80024007800F01F018E40D3
:1057F0004009800000F1E020C0F8006170BD01F0B8
:105800001F0086404809800000F1E020C0F8806158
:1058100070BD124A114001430F48001F01607047DC
:105820000D4A121D002903D0116801431160704711
:1058300011688143116070474FF0E021042804D0C3
:10584000086920F0040008617047086940F004000E
:10585000086170470000FA050CED00E080FFFF1FB3
:1058600010B59C49884209D10121042000F07DFA3D
:105870000021BDE81040042000F077BA9649884224
:1058800009D10121082000F070FA0021BDE8104084
:10589000082000F06ABA9149884209D101211020FC
:1058A00000F063FA0021BDE81040102000F05DBA5E
:1058B0008B49884209D10121202000F056FA0021AD
:1058C000BDE81040202000F050BA8649884209D136
:1058D0000121402000F049FA0021BDE8104040209D
:1058E00000F043BA8049884209D10121802000F0AC
:1058F0003CFA0021BDE81040802000F036BA7B4918
:1059000088420AD184150121204600F02EFA204653
:10591000BDE81040002100F028BA10BD10B50121EB
:10592000084600F022FA0021BDE81040012000F0F6
:105930001CBA2DE9F0410022CC7804F00F03E406F4
:1059400001D58C7823430C784FF00F0714F0FF0F2C
:105950004FF0010C1CD005680CFA02F40E882640AA
:10596000A64211D1960007FA06F825EA080503FABF
:1059700006F848EA0505CE78282E02D0482E02D037
:1059800002E0446100E00461521C082AE4D305608F
:105990000A88FF2A1ED94568002202F108060CFA7F
:1059A00006F40E882640A64210D1960007FA06F8A3
:1059B00025EA080503FA06F848EA0505CE78282EF8
:1059C00000D14461CE78482E00D10461521C082ACF
:1059D000E3D34560BDE8F0814FF6FF7101800221FD
:1059E00081700421C17070470246002092680A420B
:1059F00000D001207047806880B2704702460020C6
:105A0000D2680A4200D001207047C06880B2704757
:105A10000161704741617047002A01D00161704700
:105A200041617047C160704741F480328261816199
:105A3000826181698069704710B52D4B1A684FF6F5
:105A40008074224042EA00100843186010BD2949C2
:105A5000C8617047F0B5264C002801DAE36900E020
:105A60006368C0F30346420D120185B2C0F30157CB
:105A70009540032F07D0C2020CD50322B2409343B6
:105A800043F0706209E023F07062636823F0706392
:105A9000636002E0AB4343F0706201B12A43002827
:105AA00001DAE261F0BD6260F0BD10B58A07120F45
:105AB0000F23934021F003040D4921448C689C433B
:105AC0008C608B68904003438B6010BD0949DC31CA
:105AD0000860704700080140000C014000100140C0
:105AE0000014014000180140001C0140002001404A
:105AF0000000014000002042B448016841F001016B
:105B000001604168B24A114041600168B14A1140E8
:105B10000160016821F480210160416821F4FE01E7
:105B200041604FF41F0181607047A8490A6822F460
:105B300080320A600A6822F480220A60B0F5803F51
:105B400007D0B0F5802F03D1086840F4A02008608A
:105B50007047086840F480300860704703460020B2
:105B600059099A4A01290AD002290AD0516A03F038
:105B70001F02012393400B4200D00120704711689F
:105B8000F5E7116AF3E718B5002000904FF4A06420
:105B90003120FFF7E3FF0099491C00910099A142D1
:105BA00001D00028F4D03120FFF7D8FF08B1012040
:105BB00018BD002018BD854A116821F0F80141EA9E
:105BC000C000106070478449086070477F4B5A6876
:105BD00022F47C1208431043586070477E490866DF
:105BE00070477A4A516821F00301014351607047C0
:105BF0007648406800F00C007047744A516821F004
:105C0000F001014351607047704A516821F4E0612E
:105C10000143516070476D4A516821F4605141EA77
:105C2000C00050607047694A002903D0517A01438F
:105C300051727047517A8143517270476649D83129
:105C400008607047614A516821F440410143516046
:105C500070475E49002220310A7001F8202901288E
:105C600005D0042802D1052081F8200070470120CA
:105C700081F82000704759490860704753490A6A03
:105C800002430A627047554944390860704710B5AD
:105C90004E4A516801F00C01514B002927D00429CC
:105CA00027D0082927D00360516801F0F0010909C5
:105CB0004C4B5C5C0168E1404160546804F4E06472
:105CC000240A1C5D21FA04F48460546804F46054CE
:105CD000E40A1B5DD940C160526802F44042920B55
:105CE000404B1B1F9A5CB1FBF2F1016110BD0360D8
:105CF000DAE70360D8E7516801F47011536803F4E0
:105D00008033022404EB914133B153689B0307D5E0
:105D1000354B59430160C7E7334B59430160C3E733
:105D20002F4B59430160BFE7284A002903D051692E
:105D30000143516170475169814351617047234A62
:105D4000002903D0916901439161704791698143B2
:105D5000916170471D4A002903D0D1690143D16187
:105D60007047D1698143D1617047184A002903D037
:105D7000D1680143D1607047D1688143D1607047D9
:105D8000124A002903D0116901431161704711695A
:105D900081431161704711494039086070470E49CD
:105DA000C86470470949C87170470848416A41F0A2
:105DB00080714162704701460020044A92680A429D
:105DC00000D00120704701498872704700100240DE
:105DD0000000FFF8FFFFF6FE00004242800442424E
:105DE00000127A00D006002000093D0010B5E149FC
:105DF00088420AD101218C032046FFF7B6FF2046D6
:105E0000BDE810400021FFF7B0BFDB4988420AD14E
:105E100001214C042046FFF7B3FF2046BDE81040A7
:105E20000021FFF7ADBFD54988420AD101218C047A
:105E30002046FFF7A5FF2046BDE810400021FFF7F0
:105E40009FBFCF4988420AD10121CC042046FFF7E9
:105E500097FF2046BDE810400021FFF791BFC949D8
:105E600088420AD101210C052046FFF789FF204610
:105E7000BDE810400021FFF783BF10BD30B585B0ED
:105E800004460D46208A4CF6FF710840E98801431C
:105E90002182A0894EF6F3110840A9882A8911436E
:105EA0006A8902431143A181A08A4FF6FF4108404D
:105EB000A9890143A1826846FFF7E9FEAD48844203
:105EC00001D1039800E00298A189090408D500EBEC
:105ED000C00101EB001029684900B0FBF1F007E0B8
:105EE00000EBC00101EB001029688900B0FBF1F064
:105EF0006422B0FBF2F109010B096FF018056B4346
:105F000000EB8300A3891D044FF0320307D503EB98
:105F1000C000B0FBF2F000F00700084306E003EB1E
:105F20000010B0FBF2F000F00F000843208105B034
:105F300030BD4FF41651016000218180C180018184
:105F40000C2242818181704710B5038A4FF2FF0213
:105F500013400A884C8822438C88C9880C4322430A
:105F60001A43028210BD0021018041808180C180DE
:105F70007047002904D0818941F400518181704724
:105F8000818921F400518181704710B540F66A1370
:105F9000C1F3421301F01F040121A140012B07D0DE
:105FA000022B07D014303AB102680A43026010BDD8
:105FB0000C30F8E71030F6E702688A43026010BD43
:105FC000002A03D0828A0A4382827047828A8A43E7
:105FD00082827047028A22F00F020282028A0A43FA
:105FE00002827047828922F40062828182890A4398
:105FF00082817047002904D0818941F002018181AA
:106000007047818921F0020181817047028A22F064
:1060100020020282028A0A4302827047002904D0C9
:10602000018A41F4804101827047018A21F4804154
:1060300001827047C1F30801818070478088C0F3F6
:1060400008007047818941F0010181817047028B0E
:10605000D2B20283028B42EA012101837047028B94
:1060600002F47F420283028B0A43028370470029B5
:1060700004D0818A41F0200181827047818A21F019
:10608000200181827047002904D0818A41F01001EB
:1060900081827047818A21F0100181827047002936
:1060A00004D0818A41F0080181827047818A21F001
:1060B000080181827047002904D0818941F40041A0
:1060C000818170478189C1F30E0181817047002968
:1060D00004D0818A41F4006181827047818A21F471
:1060E000006181827047828A22F004028282828A61
:1060F0000A4382827047002904D0818A41F002015C
:1061000081827047818A21F00201818270470246B4
:10611000002012880A4200D0012070478A05C94336
:106120000180704770B5002440F66A12C1F3421333
:1061300001F01F05012606FA05F2012B0CD0022BF7
:106140000DD0838A1340090A8E40008830400BB17D
:1061500000B10124204670BD83891340F3E7038A10
:106160001340F0E740F66A120A0A01219140C94340
:106170000180704700380140004400400048004062
:10618000004C0040005000400D49086070470C4929
:10619000486070470A498860704709494AF6AA2052
:1061A0000860704706494CF6CC40086070470146CD
:1061B0000020034AD2680A4200D001207047000044
:1061C0000030004010B50120FFF7E5FDBDE81040AC
:1061D0000020FFF7E0BD2049086070471E49091FF5
:1061E000086070471C498431086070471B4A118859
:1061F00021F46071014311807047184A118821F021
:106200007F0101431180704708B5144A2C3A1044AD
:1062100000900098016008BD08B510492C39084469
:1062200000900098008808BD0B489C300068C0B200
:1062300070470A480830018841F001010180704729
:106240000548A0300068C0B2704704480830018893
:1062500041F002010180704704860D422C6C004021
:10626000384900200860091D0860091D0860091DE3
:1062700008603449344814310860704730B5314AF9
:1062800083790168002B2AD013688B431360111D9A
:106290000B680468A3430B60017911440B68046820
:1062A00023430B60274C083421680368994321601D
:1062B000231D19680568A94319604179102905D083
:1062C00011440A68006802430A6030BD2168026810
:1062D00011432160196800680143196030BD0079DD
:1062E000104402688A43026030BD002101600171E0
:1062F0000C22427181717047124910310A680243C1
:106300000A607047014600200E4A143212680A42A1
:1063100000D0012070470B491431086070470146D6
:106320000020084A12680A40064B14331B680B42CF
:1063300002D0002A00D001207047024914310860C1
:106340007047000000040140FFFF0F0010B501215D
:106350000C072046FFF714FD2046BDE81040002141
:10636000FFF70EBD21490862704720490861704758
:106370001F4A116821F0E0010143116070471B4979
:10638000A031086070471A4B1A6822F003020243DA
:106390001A601848026842F004020260012905D020
:1063A00020BF016821F004010160704730BFF8E7A9
:1063B0000F48016841F004010160016841F00201E9
:1063C00001600C48016841F00401016030BF704772
:1063D00001460020064A52680A4200D00120704758
:1063E00003490A6842EA80000860704700000E42D4
:1063F0000070004010ED00E03A4A002903D01188F7
:1064000001431180704711888143118070473548DE
:10641000001D018841F01001018070473148001DC6
:10642000018821F01001018070472E481C3000883F
:106430002C491831098840EA01407047294A010C6B
:1064400018321180111D08807047264AC0F303419D
:1064500008321180111D0880E0E7224A010C203229
:106460001180111D088070471E48103000880007F9
:10647000010B1C4814300088084370471948001D60
:1064800001888906FCD570471648001D018821F057
:106490000801018001880907FCD5704701460020EA
:1064A000104A121D12880A4200D0012070470D497F
:1064B000091D0A8882430A8070470A49091D098814
:1064C000C2B21140074A1288024202D009B101202B
:1064D0007047002070470349091D0A8882430A80DB
:1064E000704700000028004010B5FE4988420AD1DC
:1064F000C41401212046FFF738FC2046BDE81040B7
:106500000021FFF732BCB0F1804F0CD0F649884231
:1065100013D101210220FFF733FC0021BDE8104018
:106520000220FFF72DBC01210846FFF729FC0021BE
:10653000BDE810400120FFF723BCEC49884209D197
:1065400001210420FFF71CFC0021BDE810400420BD
:10655000FFF716BCE649884209D101210820FFF760
:106560000FFC0021BDE810400820FFF709BCE149FD
:10657000884209D101211020FFF702FC0021BDE86B
:1065800010401020FFF7FCBBDB49884209D10121F4
:106590002020FFF7F5FB0021BDE810402020FFF789
:1065A000EFBBD64988420AD1441401212046FFF7A7
:1065B000DCFB2046BDE810400021FFF7D6BBD049E8
:1065C00088420AD10121CC042046FFF7CEFB2046A9
:1065D000BDE810400021FFF7C8BBCA4988420AD174
:1065E00001210C052046FFF7C0FB2046BDE8104006
:1065F0000021FFF7BABBC44988420AD101214C05EA
:106600002046FFF7B2FB2046BDE810400021FFF70F
:10661000ACBBBE49884209D101214020FFF7B0FB45
:106620000021BDE810404020FFF7AABBB8498842CE
:1066300009D101218020FFF7A3FB0021BDE8104014
:106640008020FFF79DBBB34988420AD18415012100
:106650002046FFF795FB2046BDE810400021FFF7DC
:106660008FBBAD4988420AD101210C042046FFF7B7
:106670007CFB2046BDE810400021FFF776BBA74910
:1066800088420AD101214C042046FFF76EFB2046C8
:10669000BDE810400021FFF768BBA14988420AD13C
:1066A00001218C042046FFF760FB2046BDE8104026
:1066B0000021FFF75ABB10BD30B50288894C8F4DC1
:1066C000A0420DD0A8420BD0B0F1804F08D0864B2D
:1066D000984205D0854B984202D0854B984203D111
:1066E00022F070034A881A43824B984206D0824BAC
:1066F000984203D022F44073CA881A4302808A88E1
:1067000082850A880285A0420AD0A84208D0824A1F
:10671000904205D0814A904202D0814A904201D1F4
:10672000097A01860121818230BD30B5028C22F0C8
:1067300001020284028C8388048B24F0700424F00C
:1067400003050C882C4322F002020D8915434A8868
:106750002A43644DA8420BD0684DA84208D06E4D24
:10676000A84205D06D4DA84202D06D4DA8420FD170
:1067700022F008054A892A4322F004058A882A4320
:1067800023F4807323F400738D891D43CB892B433D
:1067900083800483C9888186028430BD70B5028CF1
:1067A00022F010020284028C8388048B24F4E044DB
:1067B00024F440760D884FF6FF7404EA052535432E
:1067C00022F020020E8904EA061616434A8804EADB
:1067D00002123243434EB04202D0484EB04217D16B
:1067E00022F080024E8904EA0616164326F040067F
:1067F0008A8804EA0212324323F4806323F400639C
:106800008E8904EA86061E43CB8904EA8303334358
:1068100083800583C9880187028470BD70B5028CAE
:1068200022F480720284028C8388848B24F07004AA
:1068300024F003040D88254322F400720E894FF6DC
:10684000FF7404EA062616434A8804EA0222324309
:10685000244EB04202D0294EB04217D122F4006635
:106860004A8904EA0222324322F480668A8804EAD2
:106870000222324323F4805323F400538E8904EA26
:1068800006161E43CB8904EA0313334383808583B2
:10689000C9888187028470BD70B5028C22F4805251
:1068A0000284058C8288838B23F4E04323F44076B2
:1068B0000C884FF6FF7303EA0424344325F4005593
:1068C0000E8903EA06362E434D8803EA0535354323
:1068D000044EB04202D0094EB04226D122F4804686
:1068E0008A891FE0002C014000040040000800409D
:1068F000000C004000100040001400400034014033
:10690000004C01400050014000540140001800407C
:10691000001C0040002000400040014000440140B5
:106920000048014003EA8212324382808483C9888E
:10693000A0F84010058470BD828B22F440628283EF
:10694000828B4FF6FF7303EA01210A43828370476B
:10695000F0B5048C24F480540484868B048C4FF6A8
:10696000FF7505EA013726F4734605EA0222324331
:1069700005EA03331343F74A90420ED0F64A904299
:106980000BD0B0F1804F08D0F44A904205D0F44AC1
:10699000904202D0F34A904205D124F40051394389
:1069A00041F4805104E024F402420A4342F480514D
:1069B00083830184F0BD828B22F00C028283828B60
:1069C0000A4382837047F0B5048C24F480740484F5
:1069D000858B048C4FF6FF7707EA012625F0F30537
:1069E00007EA031313432B43DA4A90420ED0DA4AE4
:1069F00090420BD0B0F1804F08D0D84A904205D0D9
:106A0000D74A904202D0D74A904205D124F400716F
:106A1000314341F4807104E024F420620A4342F4DB
:106A2000807183830184F0BD028B22F44062028373
:106A3000028B4FF6FF7303EA01210A43028370477A
:106A4000F0B5048C24F010040484068B048C4FF6FB
:106A5000FF7505EA011726F4734605EA033333434D
:106A600005EA02221A43BB4B98420ED0BA4B984219
:106A70000BD0B0F1804F08D0B84B984205D0B84B3E
:106A8000984202D0B74B984205D124F020013943F7
:106A900041F0100104E024F0A0030B4343F0100187
:106AA00002830184F0BD028B22F00C020283028B70
:106AB0000A430283704770B5048C24F001040484F7
:106AC000058B048C25F0F3054FF6FF7606EA0313D9
:106AD00013432B439F4A90420ED09F4A90420BD0C3
:106AE000B0F1804F08D09D4A904205D09C4A904218
:106AF00002D09C4A904205D124F002020A4342F09F
:106B0000010104E024F00A020A4342F00101038378
:106B1000018470BD70B505460C468E48854209D08B
:106B20008D48854206D0B5F1804F03D08B48854211
:106B300000D08B4820886188A288238958B1042816
:106B400011D0082817D02846FFF702FFE188284611
:106B5000BDE87040F0E62846FFF7ADFFE188284623
:106B6000BDE870409FE72846FFF76AFFE1882846A6
:106B7000BDE8704058E72846FFF725FFE188284622
:106B8000BDE8704017E72DE9F04107460C460025A7
:106B900001266188002900D10225A288012A00D19E
:106BA00002262088238988B13846FFF749FFE1880B
:106BB0003846FFF739FF2389324629463846FFF722
:106BC0007AFFE1883846BDE8F0416CE73846FFF7C8
:106BD00072FFE1883846FFF766FF2389324629466F
:106BE0003846FFF72DFFE1883846BDE8F0411BE746
:106BF00010B50A884B88CC881A438B8823431A43E4
:106C00000B891A434B8989891A430A43A0F8442007
:106C100010BD4FF6FF71818000210180C18041804D
:106C2000017270470021018041808180C180018113
:106C300041818181C1817047002101804180012211
:106C40008280C18001817047002101804180818064
:106C5000C1800181418181817047002904D0018870
:106C600041F0010101807047018821F0010101809C
:106C70007047002905D030F8441F41F400410180DD
:106C8000704730F8441FC1F30E0101807047002A9D
:106C900003D082890A438281704782898A43828134
:106CA0007047818270471143A0F848107047002A4E
:106CB00003D082890A438281704782898A43828114
:106CC0007047018921F0070101817047028922F094
:106CD00070020A430281704700B503461846FFF769
:106CE000F5FF188940F00700188100BD70B50D460A
:106CF00004461146602D0CD001222046FFF7DBFE32
:106D000029462046FFF7E2FF208940F00700208156
:106D100070BD01222046FFF793FEF1E730B50489EC
:106D2000E4B24FF6FF7505EA032313430B432343F5
:106D3000038130BD10B504462046FFF7EFFF2089E0
:106D400020F0070040F0070020F0700040F07000D5
:106D5000208110BD002C014000340140000400409F
:106D600000080040000C004010B504462046FFF724
:106D7000D5FF208940F480402081EAE701858282A6
:106D80007047028822F070020A430280704770B593
:106D90000589048B068C25F007050D434FF6FC4151
:106DA0000C4040F201110C4326F022064FF6FF7111
:106DB00001EA03111143314305810483018470BD4D
:106DC000028B22F070020A4302837047028B22F486
:106DD000E0424FF6FF7303EA01211143018370473C
:106DE000828B22F070020A4382837047828B22F4E6
:106DF000E0424FF6FF7303EA01211143818370479C
:106E0000002904D0018841F0800101807047018889
:106E100021F0800101807047002904D0818841F071
:106E2000040181807047818821F0040181807047CE
:106E3000002904D0818841F0080181807047818851
:106E400021F0080181807047002904D0818841F039
:106E5000010181807047818821F0010181807047A4
:106E6000028B22F008020A4302837047028B22F44D
:106E700000624FF6FF7303EA01211143018370475B
:106E8000828B22F008020A4382837047828B22F4AD
:106E900000624FF6FF7303EA0121114381837047BB
:106EA000028B22F004020A4302837047028B22F411
:106EB00080624FF6FF7303EA01211143018370479B
:106EC000828B22F004020A4382837047828B22F471
:106ED00080624FF6FF7303EA0121114381837047FB
:106EE000028B22F080020A4302837047028BC2F3B6
:106EF0000E024FF6FF7303EA01211143018370472D
:106F0000828B22F080020A4382837047828BC2F315
:106F10000E024FF6FF7303EA01211143818370478C
:106F2000028C22F002020A4302847047028C22F093
:106F300008020A4302847047028C22F020024FF6B6
:106F4000FF7303EA0111114301847047028C22F0A0
:106F500080024FF6FF7303EA011111430184704769
:106F6000028C22F400724FF6FF7303EA01211143F1
:106F700001847047028C22F400624FF6FF7303EA2B
:106F80000121114301847047028C22F400524FF614
:106F9000FF7303EA013111430184704710B50123E7
:106FA0008B40048C9C430484038C8A4013430384E9
:106FB000CFE610B504238B40048C9C430484038CDF
:106FC0008A4013430384C4E630B500F1180301245A
:106FD0008C40058CA5430584002911D008290FD0C9
:106FE000091FC1F34E001844016821F4E04101601B
:106FF00001684FF6FF7303EA02221143016030BDBE
:1070000003EB5100016821F0700101600168114338
:10701000016030BD002904D0018841F002010180E7
:107020007047018821F0020101807047002904D0D7
:10703000018841F0040101807047018821F00401BA
:1070400001807047002904D0818841F0800181804F
:107050007047818821F0800181807047028822F08A
:107060000802028002880A4302807047828822F068
:107070007002828082880A4382807047028922F0EF
:107080000702028102890A4302817047028922F0C5
:107090008002028102890A4302817047818470471D
:1070A0008185704781867047018770478187704767
:1070B000A0F840107047028822F4407202800288D3
:1070C0000A4302807047808E7047008F7047808F20
:1070D0007047B0F840007047808C7047008D704753
:1070E00002460020128A0A4200D001207047C9439C
:1070F0000182704702460020138A0B4092890A40A1
:10710000002B02D0002A00D001207047C943018221
:1071100070470000FE4A116801F038010143116018
:107120007047FB490A6822F008020A600A680243B5
:107130000A607047F6490A6822F010020A600A687D
:1071400002430A607047F248F2494160F2494160E7
:107150007047EF48EF494160EF4941607047EC48A4
:10716000016941F0800101617047E948016941F01E
:107170008001016170470420E549CA68D20701D047
:1071800001207047CA68520701D502207047C968BC
:10719000C906FBD50320704700B50346FFF7EBFF98
:1071A00002E0FFF7E8FF5B1E012801D1002BF8D1B8
:1071B000002B00D1052000BD70B505464FF43026E8
:1071C0003046FFF7E9FF042811D1D14C206940F087
:1071D000020020616561206940F040002061304676
:1071E000FFF7DAFF216941F6FD721140216170BDA0
:1071F00030B54FF430252846FFF7CEFF042810D1D4
:10720000C34C206940F004002061206940F0400038
:1072100020612846FFF7C0FF216941F6FB7211404B
:10722000216130BD00B50346FFF7A5FF02E0FFF77F
:10723000A2FF5B1E012801D1002BF8D1002B00D149
:10724000052000BD30B54FF430252846FFF7EAFF92
:10725000042810D1AE4C206940F004002061206960
:1072600040F0400020612846FFF7DCFF216941F62D
:10727000FB721140216130BD0020A549C969890711
:1072800000D50120704770B5A525FFF7F5FF00B1C7
:1072900000254FF430263046FFF77EFF042818D132
:1072A0009B4C9C48A0609C48A060206940F0200056
:1072B0002061206940F0400020613046FFF76CFFFC
:1072C00041F6EF76042805D0052802D02169314027
:1072D000216170BD206941F6DF710840206120699D
:1072E00040F0100020618D4805804FF40050FFF7FA
:1072F00053FF0528EDD021693140216170BD2DE992
:10730000F84105460E46002000904FF400573846DD
:10731000FFF742FF04280FD17D4C206940F00100A7
:1073200020612E80B8464046FFF736FFBF1E042876
:1073300004D0216939402161BDE8F881AD1C009578
:107340000099300C08804046FFF726FF216939403C
:107350002161F1E700887047F0B506460D464FF40D
:1073600000573846FFF718FF04280CD1684C2069F5
:1073700040F00100206135803846FFF70DFF21699C
:10738000BA1E11402161F0BDF0B505460E464FF41E
:1073900000573846FFF700FF042813D15C4C5D48C6
:1073A000A0605D48A060206940F0100020612E8040
:1073B0003846FFF7F1FE052804D0216941F6EF7247
:1073C00011402161F0BD2DE9F043C043C4B2C0F3C8
:1073D0000725C0F30746070E4FF400594846FFF74C
:1073E000DBFE04283CD1DFF828814A49C8F80810A0
:1073F0004949C8F80810D8F8101041F01001C8F831
:107400001010FF2C05D04548083004804846FFF78F
:10741000C3FE042807D1FF2D05D040480A3005805F
:107420004846FFF7B9FE042807D1FF2E05D03B4898
:107430000C3006804846FFF7AFFE042807D1FF2F27
:1074400005D036480E3007804846FFF7A5FE0528D0
:1074500006D0D8F8101041F6EF721140C8F810109D
:10746000BDE8F08370B505464FF430263046FFF78F
:1074700093FE042818D1264C2648A0602648A06018
:10748000206940F020002061206940F04000206128
:107490003046FFF781FE41F6DF71042805D005284C
:1074A00002D022690A40226170BD20690840206133
:1074B000206940F010002061184815B100210180BA
:1074C00001E0A52101803046FFF766FE0528EBD0DC
:1074D000216941F6EF721140216170BD2DE9F04143
:1074E00006460D4617460A4C0A48A0600A48A060A6
:1074F0004FF400584046FFF74FFE04281DD1206985
:1075000040F0100020613D43354345F0F80007E0AE
:107510000020024023016745AB89EFCD00F8FF1F33
:107520002549891C08804046FFF736FE052804D00F
:10753000216941F6EF7211402161BDE8F0811F48D9
:10754000C069800870471D48006A704700201B49C9
:107550000968890600D501207047184A002903D020
:1075600011690143116170471169814311617047CD
:1075700001460020114A012904D0D2680A4200D0F5
:1075800001207047D169C907FBD0012070470B4922
:10759000C860704704200949CA68D20701D0012099
:1075A0007047CA68520701D502207047C968C906EA
:1075B000FBD503207047000000F8FF1F00200240A9
:1075C00001684FF6FE7211400160002101604160C8
:1075D0008160C1607249724A0839904204D148689A
:1075E00040F00F00486070476D4A1432904204D159
:1075F000486840F0F00048607047694A283290427D
:1076000004D1486840F4706048607047644A3C3276
:10761000904204D1486840F4704048607047604A26
:107620005032904204D1486840F47020486070475E
:107630005B4A6432904204D1486840F4700048606C
:107640007047574A7832904204D1486840F07060E1
:1076500048607047534A111F904204D1086840F0B7
:107660000F00086070474F4A1432904204D10868F6
:1076700040F0F000086070474A4A2832904204D136
:10768000086840F4706008607047464A3C32904297
:1076900004D1086840F4704008607047414A503295
:1076A0009042FAD1086840F470200860704730B505
:1076B000026847F6F0739A430C6A8B682343D1E95A
:1076C00004452C4323438C692343CC6923434C6AF0
:1076D00023438C6A234313430360CA6842600A68E9
:1076E00082604968C16030BD0021016041608160F5
:1076F000C160016141618161C16101624162816278
:107700007047002904D0016841F001010160704711
:1077100001684FF6FE72114001607047002A03D0E5
:1077200002680A430260704702688A430260704739
:1077300041607047406880B2704702460020D10027
:1077400003D518490839096802E01549083909685C
:10775000114200D001207047C10003D51149091F13
:10776000086070470E49083948607047024600209B
:10777000D10003D50B490839096802E008490839E6
:107780000968114200D001207047C10003D50549A6
:10779000091F0860704702490839486070470000B7
:1077A00008000240080402407047162205A10FA0FD
:1077B00000F016FA11A000F013FAFEE7FEE7FEE76C
:1077C000FEE770472E2E5C53544D333246313078ED
:1077D0005F46574C69625C7372635C73746D3332DD
:1077E000663130785F69742E630000004C6F674526
:1077F00072723A2025732C2564000000486172647F
:107800004661756C745F48616E646C65722100003E
:1078100071B630480168304A01F4E06111430160FB
:10782000BFF3408FFEE7704710B52C48016841F068
:107830000101016041682A4A114041600168294AFA
:1078400011400160016821F480210160416821F448
:10785000FE0141604FF41F018160FFF7E4FF1D4905
:107860004FF00060091F086010BD10B51B4A50683A
:1078700000F00C011C4B1D4800290ED004290ED02D
:1078800008290ED003605168184AC1F30311121D74
:10789000515C0268CA40026010BD0360F3E70360F8
:1078A000F1E7516801F47011536803F48033022446
:1078B00004EB914133B153689B0307D50C4B5943FB
:1078C0000160E0E70A4B59430160DCE7064B59438E
:1078D0000160D8E70CED00E00400FA05001002405A
:1078E0000000FFF8FFFFF6FE00127A00E00600201D
:1078F00000093D0010B5A94988420AD1841401212C
:107900002046FEF732FA2046BDE810400021FEF77F
:107910002CBAA34988420AD1041401212046FEF75B
:107920002FFA2046BDE810400021FEF729BA9D49F4
:1079300088420AD1C41301212046FEF721FA2046CD
:10794000BDE810400021FEF71BBA10BD30B502881B
:1079500002F441530A884C88CD8822438C882C43FA
:1079600022430C8922434C8922438C892243CC89AF
:1079700022431A430280828B22F400628283098AA6
:10798000018230BDF0B585B005460C4602200021CD
:107990000126AA8B4FF240031A40AA8302222A84AE
:1079A000AF8BA268022A21D0A08800B102266846C7
:1079B000FEF76DF90098E188B1F5007F2CD07101D8
:1079C000B0FBF1F000EB8000A1684000B0FBF1F0EB
:1079D000401D80B20A21B0FBF1F000F00101401A15
:1079E000C0F34F004FF6FF7202EA0121821EFE2A09
:1079F00001D302200021E288084302432A84208820
:107A00006188A2890843A18811430843384340F4A0
:107A10000060A88305B0F0BD000A00EB8000A168FB
:107A20004000B0FBF1F0401D80B2D3E7002101809F
:107A300041808180C180018141818181C181072193
:107A4000018270470021018041808180C180022233
:107A5000826081817047002904D0018841F0400193
:107A600001807047018821F04001018070470029A2
:107A700004D0818B41F4806181837047818B21F434
:107A8000806181837047090901238B4099B2002AE4
:107A900003D082880A438280704782888A4382802A
:107AA0007047002A03D082880A4382807047828808
:107AB0008A43828070478181704780897047A1F531
:107AC0007E42FF3A04D0018841F480710180704702
:107AD000018821F4807101807047002904D08188D9
:107AE00041F0040181807047818821F00401818088
:107AF0007047028822F40062028002880A430280F2
:107B00007047018841F4805101807047002904D0FA
:107B1000018841F4005101807047018821F400512F
:107B200001807047012901D0008B7047808A70471F
:107B3000008A7047B1F5804F04D0018821F480415C
:107B400001807047018841F48041018070470246FE
:107B5000002012890A4200D001207047C9430181E8
:107B6000704730B50246002001F00F03012505FAE9
:107B700003F4A3B2090905FA01F4A4B291882140E3
:107B800012891A4202D0002900D0012030BD01F034
:107B90000F0201219140C94301817047003001402B
:107BA00000380040003C0040704700007CB51D4696
:107BB00016460C00009001D02044401E074B7B4429
:107BC0002A4669460190304600F03DFC05461CB14E
:107BD0000020694600F04AFC28467CBDB50800003C
:107BE0000FB4044910B503AA029800F063FC10BC5E
:107BF0005DF814FB500600200FB47CB50C0009AAF8
:107C0000009001D02044401E084B7B4469460190FF
:107C1000089800F018FC05461CB10020694600F0E9
:107C200025FC28467CBC5DF814FB000069080000B8
:107C300070B5044685690068C10601D5302600E0AC
:107C40002026C00707D070BDD4E9012130469047F7
:107C5000206A401C20626D1EF6D570BD70B50446CA
:107C600085690078C00707D170BDD4E901212020C3
:107C70009047206A401C20626D1EF6D570BD0968D1
:107C80004A0501D540B27047C905FCD500B270471E
:107C900009684A0501D5C0B27047C905FCD580B254
:107CA000704770B50C460546012A05D02878800635
:107CB00000D5EA69002302E0012305E05B1C934242
:107CC00002D2E05C0028F9D1A869E618C01AA861C0
:107CD000286A184428622846FFF7AAFF04E0D5E97D
:107CE000012114F8010B9047B442F8D32846FFF75E
:107CF000B5FF70BD2DE9F0410646002410687529D6
:107D0000314616A510D0FFF7BAFF002802DA40422C
:107D100013A507E031688A0701D512A502E04907DB
:107D200004D511A5012401E0FFF7B2FF00210A22CA
:107D300006F1240709E0B0FBF2FCB0FBF2F302FB12
:107D40001C00303078541846491C0028F3D12346D3
:107D50002A463046BDE8F04100F017BB00000000A5
:107D60002D0000002B0000002000000011680268B8
:107D7000006A530501D508700AE0D30501D50880D3
:107D800006E0130603D5C217C1E9000200E008604F
:107D9000012070472DE9FF5F15468A460446DFF84B
:107DA000AC80F8440027D8E900103E46CDE9001029
:107DB00010E03AF816106A4602A800F019FC411CBF
:107DC00007D02178890603D5E269391891420DD888
:107DD0000744761C2078800602D5E069B84205DDAC
:107DE000AE42E6DB3AF816000028E2D1A069C01BDB
:107DF000A0612046FFF71CFFD8E90010CDE9001074
:107E0000002017E03AF818106A4602A800F0F0FBCC
:107E1000B0F1FF3F81460BD000250DF1080B05E0C6
:107E2000D4E901211BF8050090476D1C4D45F7D39F
:107E300008F10100B0428046E4DB206A3844206249
:107E40002046FFF70BFFBDE8FF9F00006E420000D9
:107E500030B4002100F1240408E002F00705D20844
:107E6000303542EA4372DB086554491C52EA030587
:107E7000F3D10468002310A2250708D504F02004DC
:107E80000C4304D0C46901230CA2641EC46130BC3D
:107E900000F07BBA10B5044621461068FFF7F8FEE3
:107EA00002462046BDE810400023D1E7D21D22F053
:107EB0000701D1E90023CBE70000000030000000FB
:107EC000F0B40D460188090502D5214C7C4402E03E
:107ED0001F4C7C440E34002100F1240608E002F01F
:107EE0000F071209E75D42EA03721B097754491C28
:107EF00052EA0307F3D102780023120704D5702D4C
:107F000006D009B1022311342246F0BC00F03DBA7C
:107F100001231034F8E770B504460D462146106879
:107F2000FFF7B6FE024629462046BDE87040002312
:107F3000C6E7D21D22F00703D3E90023C0E7036898
:107F4000126843F0200303600823C3610023B7E7EE
:107F50004C4100002DE9F05F894604464FF0000ACD
:107F6000DFF874B1FB44C0F820A02046E1688847E0
:107F7000002874D0252806D0D4E901219047206A32
:107F8000401C2062F1E700265F462046E1688847F2
:107F90002028054607DB312D05D2781910F8200C72
:107FA00008B10643F1E7B00701D526F00406C4F88E
:107FB0001CA00027C4F818A02A2D09D0284601F0DB
:107FC000F8FC38B304EB8708303DC8F8185019E0C6
:107FD00059F8041B204604EB87029161E168884749
:107FE000012F054618D1E069002820DA26F0200686
:107FF0001DE0D8F8180000EB800005EB4000303899
:10800000C8F818002046E1688847054601F0D1FC11
:108010000028EED1012F0AD02E2D08D12046E1688C
:1080200088477F1C0546022F46F02006C4DBA06966
:10803000002803DA404246F00106A061F00701D0B3
:1080400026F010066C2D0BD0682D09D04C2D39D0A0
:108050006A2D35D0742D35D07A2D33D016E038E026
:10806000E1682F4620468847B842054609D16C2F63
:1080700026D04FF48060E1680643204688470546D5
:1080800004E06C2F1AD04FF4807006430DB3A5F1B5
:108090004100192802D8203546F400664A46294690
:1080A000204626604E46F8F79DF880B101280BD097
:1080B000F61D26F0070000F1080956E74020E4E726
:1080C0008020D8E70020D6E706F104094DE72846CE
:1080D00052E7206ABDE8F09FDC40000070B506461C
:1080E00000F044F90468054630460A22002100F0F9
:1080F00047FA2C6070BD401ECAB210F8011F8A42B8
:1081000002D00029F9D10020704710B5431E13F8A2
:10811000014F002CFBD105E011F8014B002C03F8B6
:10812000014B03D0521EF7D20021197010BD40EA56
:108130000103024630B59B0710D14FF0013400E037
:1081400008C208C91D1B9D4315EAC41FF8D013F0CF
:10815000FF0102F8011B0DD01B0AF8E711F8013BE3
:10816000002B02F8013B05D011F8013B002B02F86F
:10817000013BF3D130BD0022CBB210F8011B994274
:1081800000D1421E0029F8D11046704710B5431C9B
:1081900002E010F8011B71B18107FAD14FF00132F2
:1081A00002C88C1A8C4314EAC211F9D0C01A0A060C
:1081B00003D0C01E10BDC01A10BD0A0401D0801E1D
:1081C00010BD0902FCD0401E10BD421E12F8013F36
:1081D000002BFBD111F8013B002B02F8013BF9D138
:1081E0007047032A40F2308010F0030C00F0158035
:1081F00011F8013BBCF1020F624498BF11F801CBAA
:1082000000F8013B38BF11F8013BA2F1040298BF0E
:1082100000F801CB38BF00F8013B11F0030300F078
:108220000782083AC0F0088051F8043B083A51F838
:1082300004CBA0E80810F5E7121D5CBF51F8043B21
:1082400040F8043BAFF30080D20724BF11F8013B94
:1082500011F801CB48BF11F8012B24BF00F8013BF6
:1082600000F801CB48BF00F8012B704702F0FF0374
:1082700043EA032242EA024200F002B84FF0000251
:108280000429C0F0128010F0030C00F01B80CCF128
:10829000040CBCF1020F18BF00F8012BA8BF20F896
:1082A000022BA1EB0C0100F00DB85FEAC17C24BFEA
:1082B00000F8012B00F8012B48BF00F8012B704794
:1082C0004FF0000200B5134694469646203922BF6F
:1082D000A0E80C50A0E80C50B1F12001BFF4F7AFBA
:1082E000090728BFA0E80C5048BF0CC05DF804EB9C
:1082F000890028BF40F8042B08BF704748BF20F80A
:10830000022B11F0804F18BF00F8012B704710B5F9
:10831000044610F0030F08BF11F0030F40F0158062
:108320004FF0013E121FC0F20E8051F8043BA3EB48
:108330000E0C2CEA030C1CEACE1C08BF40F8043BD0
:10834000F0D0A1F1040102F10402521E08DB11F881
:10835000013B002B00F8013BF7D11146FFF78EFFE0
:10836000204610BD704770477047704700487047FF
:10837000106C002010B5FFF7F9FF006810BD10B5B4
:108380000446FFF7F3FF046010BD2DE9F0470D46EA
:1083900099469246044600F124080168880604D5EF
:1083A000E06921F01001216000E00120A84201DD18
:1083B000471B00E00027A1697A1902EB0900081A9F
:1083C000A0612078C00602D42046FFF731FC0026C9
:1083D00008E0D4E901211AF806009047206A401C01
:1083E000761C20624E45F4DB2078C0060AD5204674
:1083F000FFF71EFC06E0D4E9012130209047206AF7
:10840000401C2062381EA7F10107F4DC07E0D4E924
:10841000012118F805009047206A401C2062281EA0
:10842000A5F10105F3DC2046FFF718FC20780006D3
:1084300002D50220BDE8F0870120FBE701694A1C54
:1084400002610878704700B58FB0CDE90131002195
:10845000059105497944CDE9031011466846FFF7B7
:1084600079FD0FB000BD0000E5FFFFFF0A6802F8CC
:10847000010B0A607047D1E900239A4202D2531CD3
:108480000B601070704710B5436913B1AFF30080F3
:1084900001E0FFF706FC012010BD127800F1240175
:1084A0000A7000224A700122EDE711684FF0FF3296
:1084B000E9E70000074B70B50D467B44FFF7C3FFAB
:1084C0000446284600F011FD10B14FF0FF3070BD9A
:1084D000204670BD25B2FFFF10B5436913B1AFF35D
:1084E000008001E0FFF756FC012010BD128800F16A
:1084F000240182840022C2840122EDE711684FF03A
:10850000FF32E9E72DE9F0418046D21D22F0070253
:108510000025D2E90002F52915A614D0011E72F13A
:10852000000106DA0023D0EB030063EB020211A680
:1085300008E0D8F800108B0701D50FA602E0490724
:1085400001D50EA601251146002408F1240704E0F8
:1085500000F0ACF830323A55641C50EA0102F7D111
:108560002B46324621464046BDE8F041FFF70DBF9D
:10857000000000002D0000002B0000002000000083
:108580002DE9F04791460F4680460446002614F830
:10859000015B2DB100F082F80068405DC007F6D1A4
:1085A0002B2D02D02D2D18D0641E4A463946204668
:1085B00000F04CFC27B13968A14201D1C7F8008016
:1085C0004FF0020471050BD54042002803DDFFF790
:1085D000CDFE0460A007BDE8F08746F48066E4E7BE
:1085E0000028F8DAFFF7C2FE04606FF00040F2E7FF
:1085F00070B516460C46054600F050F8036893F82F
:108600000101012806D0FF2C0FD8185D68B10120A8
:108610002C7070BDD3F807013246214603F20713D0
:1086200003442846BDE8704018474FF0FF3070BD46
:1086300010B5203AC0F00B80B1E81850203AA0E8FD
:108640001850B1E81850A0E81850BFF4F5AF5FEA31
:10865000027C24BFB1E81850A0E8185044BF18C9E4
:1086600018C0BDE810405FEA827C24BF51F8043B8B
:1086700040F8043B08BF7047D20728BF31F8023BDF
:1086800048BF11F8012B28BF20F8023B48BF00F873
:10869000012B704700487047106C002010B500F0A7
:1086A0004DFC001D10BD00BF7516000030B5B0F1C7
:1086B0000A024FEA900E71F100034EEA817EB0EBA0
:1086C0000E0061EB91014FEA101E4EEA017E10EBA5
:1086D0000E0041EB11114FEA102E4EEA016E10EB25
:1086E0000E0041EB11214FEA104E4EEA014E10EB05
:1086F0000E0041EB1141401841F100014FEAD0005A
:1087000040EA41704FEAD10110EB80054FEA810445
:1087100044EA907444EB01046D1944EB0404521BC9
:10872000A3414FF0000348BF0A3200D530BD401CC2
:1087300041F1000130BD70472DE9FF4F0C461E4648
:108740004FF0FF378BB0D2E90001DDF860800A906E
:108750008A46C1F30A5505B93D46002108464FF047
:108760000000BAF1000F00F4400005DA00EB8000D1
:108770004FF4400101EA50004FEA9059B9F1010F5E
:1087800000DDB9460A9850EA4A000ED044F610506F
:10879000A5F2FF3545432F14B8F1000F1ED07542E6
:1087A000291E1EDDC9F100021CE0B8F1010F4FF0D7
:1087B000000001D0302103E0F24305E02154401CC9
:1087C000B042FBDB30460022002121540B99C1F856
:1087D0000880C1E900200FB0BDE8F08FBD1B6D1C03
:1087E000DEE74A4600DA694206A800F0F9FB06AB6C
:1087F00093E8070003AB83E8070050460A9900F0AE
:10880000A3FC8DE80700A0F500501F3800900398E6
:10881000002D09DD42F21F014A46084403A90390D6
:10882000684600F002FF08E0A0F500504A461F38F5
:1088300003A90390684600F00CFF8DE807000004D0
:10884000000C03D04FF0FF30410800E01046B8F1B3
:10885000000F03D00022009215461EE0751E05D4BD
:10886000FFF724FF303262556D1EF9D5B346012261
:10887000084302D000227F1C04E02078302801D178
:1088800000227F1E002A099786D01DE0112D07DAED
:10889000FFF70CFF303262556D1C50EA0102F5D132
:1088A000084302D00098C8B10EE00021681E05E020
:1088B000235C625C63542254401E491C8142F7DBF6
:1088C000AB46A81B401E0990002004F80B000B9833
:1088D000099AC0F80880C0E9002B7CE711264FF008
:1088E000000859E72DE9F04F88460446D21D22F0D2
:1088F000070191B0D1E90001CDE90A0100F0DFFFE5
:1089000002460B98C00F01D02D2007E02068810798
:1089100001D52B2002E0202101EAC000032A0990A2
:1089200001D0072A05DB03464146204600F00AFB3A
:108930000BE12078800601D5E06900E00620B8F15F
:10894000650F814606D0B8F1660F18D0B8F1670FF1
:1089500070D131E00020B9F1110F009001DB11233B
:1089600001E009F101030AAA01A90CA8FFF7E4FE3E
:10897000DDE90C70002609F10105834647E001207E
:108980004B4600904FF000470AAA01A90CA8FFF738
:10899000D3FEDDE90DB00C995D46002610B909F152
:1089A00001000D18B9EB050003D4C0F1FF3609F141
:1089B0000105A5EB09002BE0B9F1010F01DA4FF039
:1089C00001090020B9F1110F0090484601DD112383
:1089D00000E003460AAA01A90CA8FFF7ADFEDDE9F5
:1089E0000C704D4600268346207800070AD4AB451C
:1089F00000DA5D4601A8012D04DD411911F8011CC2
:108A0000302907D04F4502DA17F1040F04DA0120AC
:108A100082460FE06D1EEEE7002F02DCED1B3E44A8
:108A200003E0781CA84200DD7D1CB81B00F1010AA0
:108A30004FF000472078000703D4AA4501DB4FF030
:108A4000FF3A0021B7F1004F0DF143088DF84310B4
:108A500024D002202B23002F01DA7F422D230A216C
:108A6000021EA0F1010000DC5FB197FBF1FC97FB57
:108A7000F1F201FB1C7C17460CF1300C08F801CD1B
:108A8000EEE7A8F1010003702188090501D5452111
:108A900000E06521A0F1010800F8011C09980FA968
:108AA000A1EB0807FF1D00B10120411901EBEA709D
:108AB000A1693844081A401EA0612078C00602D47B
:108AC0002046FFF7B5F8099828B1D4E9012190476D
:108AD000206A401C20622078C00622D52046FFF77D
:108AE000A7F81EE0002E04DBB34502DD01A8805D7F
:108AF00000E03020D4E901219047206A401C206228
:108B0000761CAAF101005FEA000A0AD100F016FA09
:108B1000C0680168405CD4E901219047206A401C8C
:108B20002062281EA5F10105DCDC07E0D4E9012163
:108B300018F8010B9047206A401C2062381EA7F1EC
:108B40000107F3DC2046FFF789F8032011B043E664
:108B50002DE9F04F04460D46D21D22F0070089B0E2
:108B6000D0E9009248461746394600F0A8FE024672
:108B7000F80F01D02D2307E02068810701D52B23B2
:108B800002E0202101EAC0038DF820300BB1012062
:108B900000E00020032A824601D0072A04DB294690
:108BA000204600F0CFF93DE12078800601D40D2564
:108BB00000E0E569C7F30A560D2D49DA00214FEAB6
:108BC000175B08464FF00000002F00F4400007DA62
:108BD00000EB80004FF4400100EBD07001EA600030
:108BE0008115012901DD4FF0FF3100224FEA850C8C
:108BF000BCF1180F06D31346ACF118004FF08052A9
:108C0000C24003E04FF4801323FA0CF30CF10C0C78
:108C1000BCF1200F04D3ACF1200C09FA0CF001E0F8
:108C200007FA0CF000294FF0004801DD18B90FE0F9
:108C30000ED140450CD319EB02095F4121B94045E3
:108C400002D19F4329EA0209BBEB175F00D0761CD3
:108C50002088000502D57B48784402E079487844B2
:108C6000193808AA302302F80A30037C0AF10101FE
:108C7000002E0AF1020A53546A4602DC4FF030011A
:108C800001E04FF031014FF001088DF8001002D0E3
:108C9000A6F2FF3603E059EA470100D06A4E002DE4
:108CA00002DC2178090704D54FF002082E218DF847
:108CB0000110C44600210BE0C7F303433F01C35C2E
:108CC000491C6D1E02F80830052908F1010801DA77
:108CD000002DF1DC00210CE000EB1973491C1B781E
:108CE0006D1E082902F808304FEA091908F1010839
:108CF00001DA002DF0DC2178890602D514E0A8F114
:108D00000108E04505DD02EB080111F8011C3029DE
:108D1000F5D0B8F1000F07DD02EB080111F8011CD6
:108D20002E2901D1A8F10108002D05DD3E2102F810
:108D300008106D1E08F10108407C002E02F80800A2
:108D400008F1010804DA2D20764202F8080002E05A
:108D50002B2002F808000A214FF47A70864208F1AD
:108D600001080BDB96FBF0F3303302F8083096FB7A
:108D7000F0F308F1010800FB136601E0642E0CDB40
:108D8000642096FBF0F3303302F8083096FBF0F3E2
:108D900008F1010800FB136601E00A2E06DB96FBD2
:108DA000F1F0303002F8080008F1010896FBF1F00C
:108DB00001FB1060303002F80800A16908F10108D9
:108DC00008EB050202EB0A00081AA0612078C00631
:108DD00002D42046FEF72CFF216A08AE01EB0A0000
:108DE000206204E0D4E9012116F8010B9047BAF1A2
:108DF000010AF7D22078C00602D52046FEF718FFF8
:108E00006E4609E016F8010B3E280FD0D4E9012187
:108E10009047206A401C2062B8F10108F2D2204637
:108E2000FEF71CFF09B00320BDE8F08F206A28443C
:108E3000206203E0D4E90121302090476D1EEBD37E
:108E4000F8E700004F34000002FCFFFF2DE9F05F5F
:108E5000824615468B4600270AF10104B946007880
:108E6000302801D09DB113E014F8010B01277828B8
:108E700003D0582801D045B10AE00DB1102D07D11B
:108E8000002714F8010B102502E0082500E00A2550
:108E90000026B0460EE005FB080005FB06F10127A1
:108EA0001FFA80F801EB1046B6F5803F00D3B946B3
:108EB00014F8010B294600F085F80028EBDABBF125
:108EC000000F05D00FB1641E00E05446CBF80040FF
:108ED000B9F1000F06D0FFF749FA02210160C81E60
:108EE000BDE8F09F48EA0640FAE7007B00F080000A
:108EF00070477546FFF7CEFBAE4605006946534600
:108F000020F00700854618B020B5F7F7E7F9BDE86F
:108F100020404FF000064FF000074FF000084FF0E0
:108F2000000B21F00701AC46ACE8C009ACE8C00971
:108F3000ACE8C009ACE8C0098D46704700487047EE
:108F4000306C00202DE9F0411F46044603260168DD
:108F5000072A01F4006004DB08B116A505E016A598
:108F600003E008B115A500E015A521F01000206070
:108F7000A069C01EA0610FB1401EA0612046FEF78F
:108F800057FE4FB1D4E9012138469047206A401C72
:108F90002062C01C206206E0206AFAE7D4E90121C1
:108FA00015F8010B9047761EF8D22046FEF756FEC4
:108FB000BDE8F0814E414E006E616E00494E4600A4
:108FC000696E66003A2800D2303820F02002412A2B
:108FD00001D3A2F13700884201D34FF0FF30704730
:108FE0002DE9F047814616468AB0334878440DC8CB
:108FF0008DE80D0030487844801C03AC0DC884E82F
:109000000D0041F69B300844372190FBF1F290FBB4
:10901000F1F5A5F1800501FB12041B3C02D5644269
:10902000012000E00020DFF890A080460027FA44ED
:10903000AAF1BE0A0DE0E00709D03246684607EB08
:1090400047010AEB810100F004FB8DE80700641082
:109050007F1C002CEFD1184F7F44AC3F18E0E8078D
:1090600014D007EB04100DF1180A90E80E008AE8FE
:109070000E00C068F04201D198190890324606A946
:1090800003A800F0E6FA03AB83E807006D10641C48
:10909000002DE4D132466946B8F1000F03A802D092
:1090A00000F0C3FA01E000F0D4FAC9E90001C9F800
:1090B00008200AB0BDE8F0874C3100000446AFF349
:1090C00000802046F7F7F1F84FF0013C50F8042BF0
:1090D00051F8043B9A4221D1A2EB0C03934313EACB
:1090E000CC1317D150F8042B51F8043B9A4215D1F8
:1090F000A2EB0C03934313EACC130BD150F8042BCF
:1091000051F8043B9A4209D1A2EB0C03934313EAB2
:10911000CC13DBD04FF00000704700BFD01A01BA6B
:10912000B1FA81F101F0180122FA01F0CB40C1F14E
:109130002001DBB2C0B2C01A2CFA01F3D11A91435C
:1091400011EAC311E6D170475FEA400C08BF91F005
:10915000000F4FEA8C234FEAC12243EA51514FEAF4
:109160001C5018BF00F5F0404FEA300018BF41F026
:1091700000415FEA6C5C00F02980BCF1FF3F08BF52
:1091800040F080407047130C06BF12044FF0100CE3
:109190004FF0000C130E04BF12020CF1080C130F59
:1091A00004BF12010CF1040C930F04BF92000CF1E8
:1091B000020CD30F04BF52000CF1010C11464FF00A
:1091C0000002A0F11F00A0EB0C00704711F0004F4F
:1091D00008BF704731F000413FF4D5AF0B0C06BF1C
:1091E00009044FF0100C4FF0000C0B0E04BF0902E5
:1091F0000CF1080C0B0F04BF09010CF1040C8B0FD0
:1092000004BF89000CF1020CCB0F04BF49000CF124
:10921000010CCCF12003A0EB0C0022FA03F302FABC
:109220000CF241EA030100F10100704720F07F4C8D
:1092300080EA030023F07F47ACEB070303F57C5380
:1092400000F0004003F1FF032DE980494FEA154B80
:1092500009B44FEA144325EA0B4E24EA03480FF2FF
:10926000042606EB132749083E785FEA320203FB27
:109270000667C7F5000707FB06F64FEA54374FEAC3
:10928000D64606F1020607FB066CCCF1005C4FEAFD
:109290001C472CEA074C07FB06F40CFB06F504EB15
:1092A00015464FEA961634BF00204FF000404FEAB3
:1092B000D13706FB07FC4FEA1C4C0CFB0BF7D21B0B
:1092C00003FB0CF761EB07010CFB0EF7B0EB07405B
:1092D00072EB17420CFB08F734BFA2EB0742B2EB6C
:1092E000074261EB17414FEA0C444FEA910706FB36
:1092F00007FC4FEA1C4C0CFB0BF7B0EBC74072EBC2
:10930000573203FB0CF734BFA2EBC742B2EBC742A4
:1093100061EB57310CFB0EF7B0EBC70072EB5772E5
:109320000CFB08F734BFA2EBC702B2EBC70261EB3C
:109330005771039F4FEA816141EA921104EBCC041B
:109340004FEAD1374FEA826206FB07FC42EA9012ED
:109350004FEA80604FEA1C4C0CFB0BF7D21B03FB5F
:109360000CF761EB07010CFB0EF7B0EB074072EB5B
:1093700017420CFB08F734BFA2EB0742B2EB0742DF
:1093800061EB17414FEA8C554FEA910704EB9C249F
:1093900006FB07FC4FEA1C4C0CFB0BF7B0EBC7407D
:1093A00072EB573203FB0CF734BFA2EBC742B2EBB0
:1093B000C74261EB57310CFB0EF7B0EBC70072EB05
:1093C00057720CFB08F734BFA2EBC702B2EBC7021F
:1093D00061EB577115EB4C254FEA816141EA92111F
:1093E0004FEA82624FEAD13742EA901206FB07FC4D
:1093F00044F100044FEA80604FEA1C4C0CFB0BF771
:10940000D21B03FB0CF761EB07010CFB0EF7B0EB73
:10941000074072EB17420CFB08F734BFA2EB074280
:10942000B2EB074261EB174115EB1C154FEA813196
:1094300041EA92414FEA823242EA90424FEA80305A
:109440004FEA0C7644F1000448EA03434EEA0B4825
:109450004FF0000EB2EB080C71EB030724BF62461D
:1094600039464EEB0E0E4FF0000B001852414941A9
:109470004BEB0B0BB2EB080C71EB03077BF1000B12
:1094800024BF624639464EEB0E0E4FF0000B00181B
:10949000524149414BEB0B0BB2EB080C71EB03074C
:1094A0007BF1000B24BF624639464EEB0E0E51EAAB
:1094B000020718BF46F0010616EB0E7655F10002C2
:1094C00054F1000103D5BDE88901BDE80088BDE87D
:1094D0008901BDE80048B619524141EB0101A3F1F1
:1094E0000103704780807F7E7D7C7B7A79787776F8
:1094F00076757473727171706F6E6E6D6C6C6B6A71
:109500006A6968686766666564646363626161600E
:10951000605F5F5E5E5D5D5C5C5B5B5A5A5959588B
:1095200058575756565555555454535352525251F5
:10953000515050504F4F4F4E4E4D4D4D4C4C4C4B4B
:109540004B4B4A4A4A494949484848474747474692
:1095500046464545454444444443434343424242CE
:1095600042414141002B26D4770021D01CB54FEA5F
:10957000370703B44FF010004FF010014FF0000018
:109580000FBCBDE810400BF1010BBBF1010F08BF90
:109590005FEA170722BF12F1010211F101014FF03A
:1095A000004143F1000300F0004043EA000070472F
:1095B000F9D35708DAE746EA064613F1400F4FEAB7
:1095C00016461FDD13F1200FDFBF16430A460021A8
:1095D00020335B42C8D0C3F1200746EA064602FAB0
:1095E00007F74FEA164646EA0706C3F1200722FAB4
:1095F00003F201FA07F721FA03F14FF0000342EA00
:109600000702B1E746EA020646EA06464FEA164670
:1096100046EA0106BCBF46EA0646360C4FF0000398
:109620004FF000024FF000019EE72DE9C04893463D
:1096300030B491E8380007C831EA400C48BF34EA3A
:10964000430C03D5FFF7F2FDFFF78CFFF0BCBDE83C
:1096500000882DE9C048934630B491E8380007C827
:1096600010F0804F08BF13F0804F03D100F005F8D1
:10967000FFF778FFF0BCBDE8008820F07F4780EA64
:10968000030023F07F4C07EB0C03A3F57C5300F0A1
:109690000040A3F1FE0392F0000F00F0B38095F0BC
:1096A000000F00F077802DE901494FEA11404FEAA1
:1096B000144621EA004800FB06FC24EA064708FBA2
:1096C00006F607FB08F800FB07F718EB06484CEB1B
:1096D000164C4FEA124B18EB07484FEA15464CEB75
:1096E000174022EA0B4E0BFB06FC25EA06470EFB51
:1096F00006F607FB0EFE0BFB07F71EEB064E4CEBC8
:10970000164C4FF000061EEB074E4CEB174B18EBB8
:109710000B0840F1000018EB0E0B58EB000840F16D
:1097200000008F1A4FF000013CBFC943661B14BFF5
:10973000B5EB040C00213CBFC943F61B4FEA1744AC
:109740004EEA8E0E27EA04454FEA1C4704FB0762E7
:109750002CEA074C05FB07F70CFB05F604FB0CFC99
:1097600016EB074642EB174216EB0C4642EB1C4247
:109770001BEB060658EB0202414146EA9E0601D564
:10978000BDE80189B619524141EB0101A3F1010382
:10979000BDE801894FEA14454FEA114724EA05461E
:1097A00021EA074C05FB07F406FB07F70CFB06F163
:1097B00005FB0CFC11EB074144EB17444FEA124741
:1097C00011EB0C4144EB1C4422EA074C05FB07F269
:1097D00006FB07F70CFB06F605FB0CFC16EB074631
:1097E00042EB174216EB0C4642EB1C456A1854F14B
:1097F000000148BF7047B619524141EB0101A3F186
:109800000103704795F0000F37D04FEA11424FEA3D
:10981000144721EA024624EA074C02FB07F106FB43
:1098200007F70CFB06F402FB0CFC14EB074441EBBE
:1098300017414FEA154714EB0C4441EB1C4125EA54
:10984000074C02FB07F506FB07F70CFB06F602FBCD
:109850000CFC16EB074645EB174516EB0C4645EBA3
:109860001C42121951F1000148BF7047B61952410C
:1098700041EB0101A3F1010370474FEA14454FEAA0
:10988000114724EA054621EA074C05FB07F106FBD0
:1098900007F70CFB06F24FF0000605FB0CFC12EB81
:1098A000074241EB174112EB0C4251EB1C4148BF00
:1098B0007047921841EB0101A3F101037047490081
:1098C00050EAC12018BF04204A0D18BF40F0010023
:1098D00040F2FF72B2EB515F08BF40F00200012876
:1098E00008BF052070472DE9F0414F1E00EBC7016E
:1098F0000446D1E9000115461E4637F006020DD098
:109900002A46334600F00EFD7F1E04EBC703D3E961
:10991000002300F02FFA37F00602F1D1022F25D0F4
:10992000042F13D0062F18BFBDE8F0812A46334616
:1099300000F0F8FCD4E90A2300F01CFA2A4633466A
:1099400000F0F0FCD4E9082300F014FA2A4633466C
:1099500000F0E8FCD4E9062300F00CFA2A4633466E
:1099600000F0E0FCD4E9042300F004FA2A46334670
:1099700000F0D8FCD4E9022300F0FCF92A46334673
:1099800000F0D0FCD4E90023BDE8F04100F0F2B9CA
:10999000002213461046014900F0A8BA0000F03F2B
:1099A000012200F0E9BE002213461046114600F0E5
:1099B0009DBA30380A2801D2012070470020704734
:1099C0002DE9F04DC84A002490B0914205DA21F00B
:1099D0000043934201D805D120B110B0BDE8F04D4D
:1099E000FFF7DEBFB1F5801F1BDA53EA000209D092
:1099F000002911DA0120FEF7C2FC10B0BDE8F04DDD
:109A0000FFF7D1BF0220FEF7BAFCFFF7C1FF10B08D
:109A100081F00041BDE8F08D6FF03504362200F092
:109A2000ABFE04EB2152C1F31308B049A2F2FF339D
:109A3000414401F4801282F07F6103EB225281F0F5
:109A40004051009241EA08010022A94B00F074FD48
:109A5000044608F10200A74EC0F313000D467E44F1
:109A6000032867D2D6E90023204600F097FB1ED1D9
:109A70000098002802BFD6E9000110B0BDE8F08DC3
:109A800000F025FC07460C469B4A9C4B00F04AFC24
:109A900006460D469A4A9B4B3846214600F042FC4A
:109AA00010B032462B46BDE8F04D00F063B94FF0E0
:109AB0005532954B2046294600F034FC0022934B4A
:109AC00000F02EFD06460F4622462B46104619464C
:109AD00000F028FC32463B4600F024FC0646009885
:109AE0000F46F0B100F0F3FB80468A46824A834B72
:109AF00000F018FC32463B4600F012FD22462B4691
:109B000000F01AFD05460C467D4A7E4B4046514604
:109B100000F008FC10B02A462346BDE8F04D00F0E6
:109B20000BBD0B4610B0324620462946BDE8F04D2D
:109B300000F002BD00224FF08043204600F01AF9E9
:109B400002460B462046294600F0D0F906460F464D
:109B5000009800F0BCFBCDE9040132463B461046BC
:109B6000394600F0DFFB0C9069480C9A40440190A4
:109B700009910B46104600F0D5FB82460246654827
:109B80008B46C8F151080B4608F5D72803217844C5
:109B9000FFF7A9FE52465B4600F0C4FB0A905E4800
:109BA0000D9152465B4604217844FFF79CFE099BC9
:109BB0000C9A00F0B7FB844601980D9B40EA080818
:109BC00060460A9A00F0D6F883460891B8F1000F73
:109BD0004EDD4FF0FF322046294600F0CDFD2246F3
:109BE0002B4600F09FFB804600988A4660B3DDE973
:109BF0000401414A414B00F095FB099100905A46FF
:109C000040465146089B00F0B5F832463B4600F00E
:109C100089FB099B009A00F0ADF84246534600F0DC
:109C20007FFC22462B4600F087FC04460D46DDE90A
:109C30000401334A334B00F075FB10B022462B462B
:109C4000BDE8F04D00F078BC5A464046089B00F055
:109C500091F832463B4600F065FB4246534600F021
:109C60005FFC10B022462B46BDE8F04D00F058BC1A
:109C7000009840B3DDE904011F4A204B00F052FB7D
:109C800080468A465A4620462946089B00F054FCE6
:109C900032463B4600F046FB4246534600F04CFC41
:109CA00022462B4600F048FC04460D46DDE904013F
:109CB000134A144B00F036FB10B022462B46BDE889
:109CC000F04D00F039BC0B465A462046294600F0BC
:109CD00033FC32463B4600F025FB10B022462B46B3
:109CE000BDE8F04D00F01CBC0000F07F645F09008F
:109CF0000000F03F2E260000763C7935EF39EA3D32
:109D00000000E0FE422EE63F5555D53F0000E03F03
:109D100086EBF9FFC6240000C424000010B500291A
:109D20000AD00878002807D005487844FFF7CCF916
:109D3000002801D0002010BD0248784410BD00006A
:109D40004A2800004228000010B500290AD00878EF
:109D5000002807D005487844FFF7B6F9002801D05D
:109D6000002010BD0248784410BD00002E290000DC
:109D70002629000010B591EA030F48BF83F0004385
:109D800000F1E283841A71EB030C05D2121943EB44
:109D90000C03001B61EB0C01DFF824E14FEA1154C6
:109DA000A4EB135C1EEA430F18BF9EEA445F73D016
:109DB00023EA0E03DCF1200E21EA045143F4801360
:109DC00032D322FA0CFE10EB0E0023FA0CFE41EB0C
:109DD0000E01CCF1200E03FA0EFE10EB0E0051F135
:109DE0000001B1F5801FCCF1200E32D201EB0451FD
:109DF00012FA0EF2BDE8104058BF7047401C38BF41
:109E00005FEA420218BF7047002814BF20F001002B
:109E100041F100014FEA410313F5001F38BF7047BD
:109E2000A1F1C04100F076BB012A43EB0302ACF183
:109E3000200CDCF11F0E32BF4FF0000E23FA0CF3A2
:109E400010EB030041EB0451B4EB115FD0D0A1EB58
:109E5000045101F5801149085FEA300001EB04511B
:109E60000ED350F1000038BF12FA0EFE08D1BDE843
:109E70001040C9E7401C38BF5FEA4202CAD1C3E7BD
:109E8000BDE810404FEA410313F5001F38BF70478B
:109E9000A1F1C04100F03EBB9EEA445F08D011EA48
:109EA0005E0FBDE8104004BF01F000410020704784
:109EB000BDE8104070B500F0DFFA00BF64FBBE3EA5
:109EC0000000E0FF02494FF0000000F023BC00BF9B
:109ED0000000F87F491058BFC1F140415B1058BFE6
:109EE000C3F140438B42EFF3008070472DE9C0413E
:109EF00030B4DFF8A0C23CEA111418BF3CEA1314D6
:109F000000F0EC8081EA03051CEA111444EAD574E0
:109F100018BF1CEA131500F0C780A4EB05044FF02E
:109F2000004545EAC12145EAC32341EA505143EACD
:109F3000525304F17F74994204F500344FEAC02073
:109F40004FEAC22208BF904200F09C804FEA13659E
:109F50000FF24016765D4FEA134506FB05F7C7F191
:109F6000807706FB07F74FEAD737A7FB03687642EF
:109F7000C8F58038A7FB06CE38BFA8F1010807FB5B
:109F800008E64FF0000EA6FB028CE6FB03CEDCF1E8
:109F9000000CCEF1004E38BFAEF1010EA6FB0C58FE
:109FA0004FF000074FF00005E6FB0E87A1FB08C647
:109FB000A0FB07CE16EB0E0645F10005E1FB076599
:109FC00015F1E04E7EBFA4F580345FEA46066D4190
:109FD00016F1800745F100054FEA17274FEA06669C
:109FE00047EA0567A6F1DE46B6F1805F4FEA152520
:109FF0001FD9384624F0010C05EBC471BCF1FE6F8B
:10A0000001EB0C1102D8F0BCBDE8008124425CBF1A
:10A0100001F5801E9EEAC47F02D4F0BCBDE8008139
:10A02000244238D4F0BCA1F1C041BDE8004100F0A9
:10A0300071BA4FEAD22242EA43524FEAD323A7FB36
:10A0400002864FEAD02040EA415007FB03661EEA31
:10A050000E0F4FEAD12105FB026658BFA6EB005652
:10A06000B6EB00564FEA520E4EEAC37E18EB0E0EC8
:10A0700056EB530EBDD518EB02085E417F1C55F11F
:10A080000005B6E74FF480154FF000074FF00006CB
:10A090004FF00008ADE7F0BC4FF0000001F1C04107
:10A0A00001F00041BDE8008111EA0C1F0CEA131514
:10A0B00000D00CE013EA0C1F00F025804FF00000E8
:10A0C000F0BC81EA030101F00041BDE80081F0BC71
:10A0D000BDE8004181EA030100F01CBAF0BCBDE814
:10A0E000004170B500F0C8F9097EFC3E00F007B8E9
:10A0F00081EA03014FF0000001F00041704781EA5E
:10A10000030100F007BAF0BCBDE800414FF00000C9
:10A1100021497047FFFDFBF9F7F5F4F2F0EEEDEBA6
:10A12000E9E8E6E4E3E1E0DEDDDBDAD8D7D5D4D355
:10A13000D1D0CFCDCCCBCAC8C7C6C5C4C2C1C0BFA1
:10A14000BEBDBCBBBAB9B8B7B6B5B4B3B2B1B0AFA7
:10A15000AEADACABAAA9A8A8A7A6A5A4A3A3A2A18B
:10A16000A09F9F9E9D9C9C9B9A9999989797969546
:10A1700095949393929191908F8F8E8E8D8C8C8BE2
:10A180008B8A89898888878786858584848383826A
:10A19000828181800000FF070000F87F51EA030CF4
:10A1A00017D41CF5801F58BFBCF5801F00F1068036
:10A1B000994218BF704708BF9042704707D711F502
:10A1C000801F58BF13F5801F19D4994270478942E8
:10A1D00070471CF5801F08D5BCF5801FF7D58B4252
:10A1E00018BF704708BF824270474FF4001C1CEB39
:10A1F000410F38BF1CEB430F01D28B42704770B543
:10A2000000F03AF9922449004FF000514FF080538A
:10A21000FFF760BE4FEA41034FEA5353A3F5806353
:10A22000D3F11E03C8BFD3F1210C0CDD4FF0004267
:10A2300042EAC12242EA505232FA03FC8CEAE17C43
:10A24000ACEBE1707047102BC4BF0020704703F5E2
:10A25000787CBCF1FF3F04D06FF0004282EA21001D
:10A26000704770B500F008F94992248000207047CB
:10A27000F2E700004FEA1153A3F58063D3F11E0308
:10A28000A8BFD3F1200C08DB4FF0004242EAC12204
:10A2900052EA505232FA03F0704709420BD4102BA5
:10A2A000C4BF0020704703F5787CBCF1FF3F05D0A8
:10A2B0004FF0FF3070474FF00000704770B500F06E
:10A2C000DBF800BF4992248000207047F0E710F0CF
:10A2D000004248BF4042B0FA80F310FA03F10AD0BE
:10A2E000C3F11D0303F580634FEA415002EB0352B3
:10A2F00002EBD12170474FF000007047B0FA80F3B5
:10A3000010FA03F10AD0C3F11D0303F580634FEA8D
:10A3100041504FEA035202EBD12170474FF0000049
:10A3200070470000DFF848C170B51CEA111E1EBF5F
:10A330001CEA13159EEA0C0F95EA0C0F00F06F80D3
:10A3400081EA030423EA4C134EEAD47E21EA4C113D
:10A3500041F4801143F48013AE44A1FB024CA0FBF6
:10A360000365AEF17F7E361955EB0C05A1FB034C5E
:10A370004CF10003A0FB021C16EB0C06654153F1E7
:10A380000003094218BF46F0010613F4007F0BD109
:10A390004FEA03314FEA0530340341EA155140EAF0
:10A3A00016506FF003020AE04FEAC3214FEAC520BE
:10A3B000F40241EA555140EA56506FF0020202EBB6
:10A3C0002E4201EB025585EACE710AD05FEA440CB9
:10A3D00018BF24F0004450F1000041F1000120EAD0
:10A3E000D47040F2FE7C624500D270BDA84214BF1A
:10A3F0004FF080444FF04044002E08BF0024BEF1CF
:10A40000806FA8BFA1F1C041BDE8704080F282809A
:10A410004FF0000001F1C04101F0004170479EEA99
:10A420000C0F0CEA131518BF95EA0C0F06D04FF06D
:10A43000000081EA030E0EF0004170BD00F01CF830
:10A440008900013E00F007B800F009B84FEA430C5C
:10A450005FEA5C5C08D081EA030100F05BB84FEA78
:10A46000410C5FEA5C5CF6D14FF000000149704797
:10A470000000FF070000F87F0EF1020E2EF0030E21
:10A480005EF8046B364205D4012A43EB030515F54B
:10A49000001F12D8012841EB010C1CF5001F0CD83D
:10A4A0000ED14FEAD17C15F5001F0CEB4C0C0CF1D2
:10A4B000020C08BF4CEBD37C04E04FF0080C01E029
:10A4C0004FEAD37C0CEB4C0526FA05F606F007069E
:10A4D000B6F1040C06D20EEB860CBDE870404CF0D1
:10A4E000010C6047DFE80CF0090B02024FF000415D
:10A4F0004FF00000A1F5002170BD1946104601285B
:10A5000051EB010418BFD4F5001484BF002001F002
:10A51000004170BD0808A0F500114FEA31017047F5
:10A5200091EA030F10B581F000413FF52BAC83F0A9
:10A53000004300F009B8000010B591EA030F48BFCE
:10A5400083F000433FF51EAC841A71EB030C07D275
:10A5500012198CF0004C43EB0C03001B61EB0C0157
:10A56000DFF8A4E14FEA1154A4EB135C1EEA430F99
:10A5700018BF9EEA445F00F0B08023EA6E035242A7
:10A5800021EA0451C3EB6E0338BF5B1EDCF1200EE1
:10A5900025D322FA0CFE10EB0E0043FA0CFE41EB21
:10A5A0000E01CCF1200E03FA0EFE10EB0E0051F15D
:10A5B0000001CCF1200E29D412FA0EF201EB045165
:10A5C000BDE8104058BF7047401C1CBFB2F1004F9F
:10A5D000704700280CBF491C20F00100704712EBA7
:10A5E000020E43EB030218BF4FF0010E4EEA420287
:10A5F000ACF1200CDCF11E0E54D943FA0CFE10EB2A
:10A600000E0051F1FF31CCF11E0ED5D50EF1010E29
:10A6100012FA0EFE404141EB010101EB445C5FEA9E
:10A620005C5C10D910EBDE7001EB045138BFBEF159
:10A63000004FBDE8104018BF704700280CBF491CF0
:10A6400020F00100704730D24FEAD42C11F50011F0
:10A6500024F400641BD0B1FA81F20B3AA41AA41EB0
:10A66000D2F12003914030FA03F31943904001EBFB
:10A67000CC71002C01EB0451BDE81040A8BF70471D
:10A6800001F1C0414FF0000001F000417047B0FA05
:10A6900080F310FA03F100D110BDE41A173C48050D
:10A6A000C90AE4E701EB045110BD491001EB045164
:10A6B000BDE810404FEA300002E04FF00001704763
:10A6C0004A0008BF0042F8D0B2F5001F28BF70470B
:10A6D00001F000414FF0000070479EEA445F07D050
:10A6E00011EA5E0FBDE8104004BF00210020704752
:10A6F000BDE8104070B5FFF7BFFE00BF40DFF63E7B
:10A7000083F00041104670470000E0FFFEF7EAB812
:10A71000FEF71EBA0CF00F03092B08BF082000F04B
:10A7200059800A2B0BD0082B18BF704708BF1CF0AC
:10A73000400F0AD04FF000004FF0000170471CF0AE
:10A74000400F18BF4FF0004070471CF0100F08D0AA
:10A7500020F0704300F07F4242EAD3014FEA437099
:10A76000704700F0604021F07F4242EA000201F0B1
:10A770007F4040EA727070474FF0FF0C4CF4E06C81
:10A780001CEA11531CBF9CEA030C9445C2BFDA4279
:10A7900001EB02517047002B0DD0BCF1000F0FD020
:10A7A000002A01F00041A4BF41F0E04141F07F6187
:10A7B0004FF00000704701F000414FF0000070477B
:10A7C00050EA01334FF09B0C18BF4CF0806C7FF4C3
:10A7D00079AB70471CF4801F11D01CF4E02F03D01C
:10A7E0006FEACC31490070474FF04050EFF30082E0
:10A7F00022F0704242EA000282F3008870474FF074
:10A80000000070470103070F1FFFFF1F0F07030121
:10A810000000000000E0E00000FCFC000000000080
:10A820000000000000000000003F3F00003838003A
:10A83000003F3F00003F3F00003F3F00000000009E
:10A84000000000000000F808E8E8E8E80808E8E888
:10A85000E8E80808E8E8E8E80808F820E000000070
:10A860000000000000001F1017171717101017170F
:10A87000171710101717171710101F0407000000E4
:10A8800000000000C05F5555D5755555555FC00097
:10A890000809090B0505050B09090000EACC0011A0
:10A8A000F200FC2424E41FE485660000070A070088
:10A8B000020B0403040E00B3CF0012D2FE5190121B
:10A8C0002400FF80800001000F00000101010F0043
:10A8D0000000BFC6008888FF4824E4243F24E40425
:10A8E0000000080F000808050205080800BCBC00AD
:10A8F0000000000000000000000000000000000058
:10A9000000003636000000000000000000000000DB
:10A91000A3BA0000000000000000000000000000DA
:10A920000000000000583800000000000000000097
:10A93000000000A3AC0000000000000000000000C8
:10A94000000000000000000018242418000000008F
:10A95000000000000000A1A300000000FE000000B5
:10A9600000000000000000000000000033000000B4
:10A97000000000000000000000A3A1000000383427
:10A980000282C27C380000000000000000000000CD
:10A99000003737000000000000000000A3BF0000E7
:10A9A0008080BEAAAAAAEAAAAAAABE808000000441
:10A9B0008584945C54272424544C4484050400EA80
:10A9C000CC004042CC0000F888888808FF0809CAFB
:10A9D000080000003F90681F10209F402718264164
:10A9E000F000B3CF002424A4FEA3220022CC000058
:10A9F000FF00000000080601FF0001040404040435
:10AA0000FF02020200BFC600101010FF109008885D
:10AA10008888FF88888808000444827F01808040FD
:10AA2000432C102846818000BCBC001010FF109001
:10AA300000FE5252D25252525E000042827F81404A
:10AA4000308F929392FE9293968000CED5000000B4
:10AA50002424242424FC2222222322000000020297
:10AA600002020242827F0202020202020200CAD6EF
:10AA7000000000F010101010FF10101010F0000077
:10AA80000000000F04040404FF040404040F000089
:10AA900000D6D000000000000001E21CE000000031
:10AAA00000000000804020100C03000000030C3068
:10AAB00040808000C8EB0000FE0222428272022227
:10AAC00042827202FE000000FF100806010E10080C
:10AAD00006014E807F0000CDF800404042CC0004CB
:10AAE00044645C47F444444404000040201F204474
:10AAF000444444447F4444444400C1AC001010101A
:10AB0000FF1050445465C6446454444000044482D9
:10AB10007F0182824A562322524E820200BDD30018
:10AB20000000FE222222FE00FE828292A29E0000EF
:10AB300080601F0242827F00FF402F102C43800064
:10AB4000B7FE00000090884C57A42454548C840015
:10AB500000000001018042221A07024282423E01A7
:10AB6000010100CEF10080809E9292929EE0809E34
:10AB7000B2D2929E80000808F4949292F10001F201
:10AB8000929494F80800C6F7001060028C00080840
:10AB90000809FA08080808000004047E0140404142
:10ABA00041417F414141414000D7A200808080FE69
:10ABB0008282FE8080FE8282FE8080000080403F94
:10ABC00000407F80601F40807F000000B2E10000F5
:10ABD00000F8888888880808FF08090AC8080080E3
:10ABE000601F0010201F80402116182641F800B376
:10ABF000C900080808F80808081010FF101010F025
:10AC000000001030101F088848300E014080403F7F
:10AC10000000B9A6000040301E101010FF101010E8
:10AC2000101000000081814121110D0301030D115D
:10AC30002141818100CAA70000FE02FA02FE4020E5
:10AC4000D8171010F01010008047300F10678040A8
:10AC50002116081621408000B0DC00080889EA1897
:10AC600088000404FC040404FC0000020100FF014D
:10AC700086402018074080403F0000B3F5001010C8
:10AC8000F01F10F00040E05847405060C0004022E4
:10AC9000150816210000FE42424242FE0000CABCD6
:10ACA00000008060F807000000FF4020100804004A
:10ACB00000010000FF000402013F40404040407896
:10ACC00000BBAF00040444C44F4444C424242FB444
:10ACD0002404040040442424150C04FE040C152410
:10ACE00024444000B2CB000000F8494A4C48F848E0
:10ACF0004C4A49F800000010101312121212FF12F1
:10AD000012121213101000B5A500404042CC0000F2
:10AD1000FC24A4242222A36200000040201F20580B
:10AD200047504845424548504000B7B5000000FE36
:10AD30000202F2121212F20202FE00000000007F74
:10AD40002020272424242720207F000000BBD800B7
:10AD5000000022322AA6A26221110981010000000E
:10AD6000004222130B42827E02020A122346000096
:10AD7000CFB5002030AC63300088C8A8998E88A871
:10AD8000C8880022672212128040300F00003F4026
:10AD9000407100CDB3008080848484FE82838280F1
:10ADA000FF808080800000804020180700000000A5
:10ADB000FF0000000000C9FD002030AC633000023D
:10ADC00002FE0202625AC6000022672212124030BE
:10ADD0008F80432C102C438000BCB60008C8B88F6D
:10ADE000E8888840300FC8082818000008180808AC
:10ADF000FF048440300E010E30408000C8ED00009A
:10AE00008060F80780601C1010FF10101000000117
:10AE10000000FF000202020202FF0202020200BC66
:10AE2000FE00004042445840407F40405048C60029
:10AE30000000004044444444444444444444FF002B
:10AE40000000B5B1000808E8292E28E80808C80C59
:10AE50000BE80808000000FF0949897F00000F4047
:10AE6000807F000000C7B00000FE20203F2000FCD3
:10AE700024E4242223E20000807F0101FF80601F80
:10AE80008041261826418000B0E600001010101006
:10AE9000D030FF30D010101010000010080402094C
:10AEA0000808FF0808090204081000B1BE008080ED
:10AEB00080BEA2A2A2A2A2A2A2BE808080000000A8
:10AEC0000006050404044484443C00000000BAC5A4
:10AED00000404042CC0040A09E8282829EA0202062
:10AEE000000000003F908840432C1028464180809D
:10AEF00000C9E800809090484C57242424544C44C6
:10AF000080808000000000FF4949497F494949FF8E
:10AF100000000000B1B800008060F807000424249D
:10AF200025262424240400010000FF000000F94924
:10AF300049494949F90000D0C500000000FC5454BB
:10AF40005655545454FC0000000040300003394171
:10AF500041455941417300083000CFA20000000074
:10AF60007F494949494949497F0000000081412101
:10AF70001D214181FF8989898989818100CAC70092
:10AF800000028282422212FA0622224242820000FB
:10AF9000010100FC44444445444444FC00000100D9
:10AFA000B7F1000010109010101116101010D010F2
:10AFB00010000040404040435C4040504C43404003
:10AFC000404000C1A20000FE92929292FE0000FE5C
:10AFD000020202FE0000003F20100A04180000FFD9
:10AFE000000408070000BCB400003E22E2223E003C
:10AFF00010885724548C000000407E403F222200DD
:10B0000001FE424242FE010100C2B700001088C4A6
:10B010003380824222121A2622408000020100FF61
:10B0200000404242427E424242424000BEB60040A0
:10B030004424A4948C84FF848C94A4244440004031
:10B0400040405F4A4A4A4A4A4A4A5F40404000B24A
:10B05000E900101010FF10902020FF201011961012
:10B0600000000444827F01004020130C142241F8A8
:10B070000000D5D20040445465C664544400FC44EA
:10B0800044C442400020124A827F020A92601F009C
:10B0900000FF000000D0C20000FE0212929292FE59
:10B0A0009292921202FE000000FF40405F48484822
:10B0B00048485F4040FF0000B9CC00008060F807BE
:10B0C00080601C1010FF1010100000010000FF0035
:10B0D0000202020202FF0202020200BCFE0004148D
:10B0E000A444AF14040404F40F24440404001249DB
:10B0F00084423F8141310D030D3141818100BBF11B
:10B10000000202FE929292FE0206FC040404FC007D
:10B110000008180F080804FF0484402718274080FF
:10B1200000C8A100008060F807000424242526241C
:10B1300024240400010000FF000000F949494949A6
:10B1400049F90000D0C500000000FC545456555485
:10B150005454FC000000004030000339414145597F
:10B1600041417300083000CFA2000040301E101093
:10B1700010FF101010101000000081814121110DEE
:10B180000301030D112141818100CAA70000FE02C5
:10B19000FA02FE4020D8171010F01010008047303F
:10B1A0000F106780402116081621408000B0DC0097
:10B1B0001010D0FF9010804828090E0828488800F9
:10B1C000040300FF00018080432C102C438080008A
:10B1D000D0A30002FA8282FE804020504C434C50A3
:10B1E00020400008184884443F404458414E60586D
:10B1F000474000D1E900000202C2020202FE828240
:10B200008282820200004040407F4040407F4040B8
:10B21000404040404000D5FD00080888C8380C0B6D
:10B220000808E8080808080800020100FF4041413A
:10B2300041417F414141414000D4DA000202020213
:10B240000202FE020242820202020200000000002C
:10B250000000FF000000000106000000CFC20090C7
:10B260009494F49F9494941010FF1012D410002022
:10B27000262524FE141414804027182641F000D4FB
:10B28000D8004042CC0000445454547F5454544499
:10B29000400000007F201000FF15151555957F0018
:10B2A0000000C7EB00804020180F88780808F808D5
:10B2B0000808F80000001008844221100806014028
:10B2C00080403F0000CEF00000FC2024A8FFA8240E
:10B2D00000FC4444C4424000003F2221202F20A310
:10B2E000601F0000FF000000B6CF000000F8888853
:10B2F0008888FF88888888F800000000001F0808F8
:10B3000008087F888888889F80F000B5E7000000E3
:10B3100000F112141010101412F10000000040305F
:10B320000003394141455941417300083000D7DCE1
:10B3300000402010EC27242424E40404FC00000036
:10B34000000000003F4242424243444847407000F0
:10B3500000B0FC0090523410FF10345280708F08FF
:10B3600008F80800829A566322528E008040330CFF
:10B3700033408000CAFD0080828282828282E2A203
:10B38000928A8682808000000000000040807F005A
:10B3900000000000000000D7D30000FE92929292BD
:10B3A000FE0000FE020202FE0000003F20100A0420
:10B3B000180000FF000408070000BCB400000830BB
:10B3C00000FF008884532212CA0600000004040211
:10B3D00001FF00020A1242827F02020200BDAB009E
:10B3E000404042CC00202222A262222222200000E1
:10B3F0000040201F20444E4544444445464C4000F4
:10B40000D4CB00001088C4330040424242C24242C2
:10B41000424000020100FF0000000040807F000069
:10B42000000000D0D000101010FF1090001010FF8E
:10B430001010F00000000444827F018040211A07B0
:10B4400018003F40F000D6B400001088C43300401C
:10B45000424242C24242424000020100FF0000005C
:10B460000040807F0000000000D0D0000000FC04FD
:10B4700044840425C604040404E4040040300F405E
:10B4800040414E404063504C43404000D3A6000032
:10B4900010089493929292929A9690F00000004035
:10B4A00030047484848CB4848484E407106000BC09
:10B4B000B1002424A4FE2322003E22222222223E86
:10B4C0000000080601FF0106404949497F494949F2
:10B4D0004100B3CC000000FC04040414155694543D
:10B4E000341404040040300F0001010141817F0148
:10B4F0000101050300D0F20000E000FF10200888E1
:10B50000780F08E808088800010000FF00100C838D
:10B510004423180718628100BBD600201008F75496
:10B52000545454545454F404040000809090494DF1
:10B5300057252525554D4580808000B8B400101052
:10B54000D0FF9014E4AFA4A4A4AFE404000004036B
:10B5500000FF00894B2A1A0E1A2A4B888000C4A3C8
:10B5600000101090909090901010FF101011161075
:10B5700000002060203F10101000030C102040F845
:10B5800000CABD0000080808080809FA08080808E9
:10B5900008080000404041414141417F4141414153
:10B5A00041404000D6F7004044C444444440101099
:10B5B000FF101010F00000103C131014B840300EB3
:10B5C000014080403F0000B6AF00101010FF101087
:10B5D0005020D8171010F0101000007F2121217F7B
:10B5E00080402116081621408000B9CA0000FE02E2
:10B5F00022DA0610D2565A535A56D2100000FF08CB
:10B6000010080710171515FD1515171000D5CF00D8
:10B6100002FE9292FE0200101116F01413100000A8
:10B62000101F0808FF048141310D030D31418100D5
:10B63000C1AA00000022322AA6A2622111098101BA
:10B64000000000004222130B42827E02020A1223F3
:10B65000460000CFB5000000FE0202020202020214
:10B6600002020202020080601F00000000000000D1
:10B67000000000000000B3A700102C2424A4A4653F
:10B68000A624242424A4340C00404949292414521B
:10B69000897F040A1110202000BCD20000000000A5
:10B6A00000000000002F0000000007000700001449
:10B6B0007F147F1400242A7F2A1200626408132357
:10B6C00000364955225000000503000000001C22EE
:10B6D0004100000041221C000014083E081400082C
:10B6E000083E0808000000A06000000808080808DC
:10B6F000000060600000002010080402003E514974
:10B70000453E0000427F4000004261514946002111
:10B7100041454B31001814127F100027454545392B
:10B72000003C4A4949300001710905030036494986
:10B73000493600064949291E00003636000000003F
:10B74000563600000008142241000014141414148A
:10B750000000412214080002015109060032495933
:10B76000513E007C1211127C007F49494936003E4F
:10B7700041414122007F4141221C007F494949410A
:10B78000007F09090901003E4149497A007F080804
:10B79000087F0000417F4100002040413F01007FC1
:10B7A00008142241007F40404040007F020C027F8D
:10B7B000007F0408107F003E4141413E007F09099F
:10B7C0000906003E4151215E007F091929460046C5
:10B7D000494949310001017F0101003F4040403F9C
:10B7E000001F2040201F003F4038403F00631408E6
:10B7F00014630007087008070061514945430000C1
:10B800007F41410000552A552A55000041417F00E3
:10B8100000040201020400404040404000000102D8
:10B820000400002054545478007F484444380038C1
:10B830004444442000384444487F00385454541849
:10B8400000087E0901020018A4A4A47C007F08045B
:10B8500004780000447D4000004080847D00007F2B
:10B86000102844000000417F4000007C0418047848
:10B87000007C0804047800384444443800FC242444
:10B8800024180018242418FC007C0804040800482C
:10B890005454542000043F444020003C4040207C4D
:10B8A000001C2040201C003C4030403C004428103C
:10B8B0002844001CA0A0A07C004464544C441414F0
:10B8C0001414141400000000000000000000000028
:10B8D00000000000000000F800000000000000333D
:10B8E0003000000000100C06100C060000000000E4
:10B8F0000000000040C07840C0784000043F0404CD
:10B900003F040400007088FC08300000001820FF8D
:10B91000211E0000F008F000E018000000211C03C8
:10B920001E211E0000F00888700000001E21232444
:10B930001927211010160E00000000000000000062
:10B9400000000000000000E01804020000000007F2
:10B950001820400000020418E000000000402018F9
:10B9600007000000404080F0804040000202010FCC
:10B9700001020200000000F0000000000101011FB0
:10B9800001010100000000000000000080B0700014
:10B9900000000000000000000000000000010101A4
:10B9A0000101010100000000000000000030300033
:10B9B000000000000000000080601804006018060D
:10B9C0000100000000E010080810E000000F102047
:10B9D00020100F00001010F8000000000020203F91
:10B9E000202000000070080808887000003028241B
:10B9F00022213000003008888848300000182020BC
:10BA000020110E000000C02010F8000000070424E0
:10BA1000243F240000F80888880808000019212025
:10BA200020110E0000E0108888180000000F11207F
:10BA300020110E0000380808C83808000000003F38
:10BA4000000000000070880808887000001C222197
:10BA500021221C0000E010080810E0000000312244
:10BA600022110F00000000C0C000000000000030E4
:10BA70003000000000000080000000000000806036
:10BA800000000000000080402010080000010204B7
:10BA9000081020004040404040404000040404049E
:10BAA000040404000008102040800000002010085A
:10BAB00004020100007048080808F000000000308F
:10BAC00036010000C030C828E810E000071827241D
:10BAD00023140B000000C038E0000000203C2302CB
:10BAE0000227382008F8888888700000203F20202E
:10BAF00020110E00C0300808080838000718202060
:10BB00002010080008F808080810E000203F202056
:10BB100020100F0008F88888E8081000203F202037
:10BB20002320180008F88888E8081000203F20002B
:10BB300003000000C0300808083800000718202063
:10BB4000221E020008F808000008F808203F210122
:10BB500001213F20000808F8080800000020203FCD
:10BB60002020000000000808F8080800C08080803D
:10BB70007F00000008F888C028180800203F200136
:10BB80002638200008F8080000000000203F202090
:10BB90002020300008F8F800F8F80800203F003FA7
:10BBA000003F200008F830C00008F808203F2000BF
:10BBB00007183F00E01008080810E0000F102020D0
:10BBC00020100F0008F808080808F000203F2101A5
:10BBD00001010000E01008080810E0000F182424FC
:10BBE00038504F0008F8888888887000203F20006F
:10BBF000030C302000708808080838000038202125
:10BC000021221C00180808F8080818000000203F2E
:10BC10002000000008F808000008F808001F202095
:10BC200020201F000878880000C838080000073866
:10BC30000E010000F80800F80008F800033C0700B7
:10BC4000073C0300081868808068180820302C031F
:10BC5000032C30200838C800C83808000000203FF6
:10BC60002000000010080808C838080020382621E5
:10BC700020201800000000FE020202000000007FE9
:10BC800040404000000C30C00000000000000001F7
:10BC90000638C00000020202FE00000000404040E2
:10BCA0007F00000000000402020204000000000007
:10BCB0000000000000000000000000008080808084
:10BCC000808080800002020400000000000000006C
:10BCD0000000000000008080808000000019242205
:10BCE00022223F2008F8008080000000003F112041
:10BCF00020110E000000008080800000000E112046
:10BD000020201100000000808088F800000E112023
:10BD100020103F200000808080800000001F222231
:10BD200022221300008080F0888888180020203F9D
:10BD3000202000000000808080808000006B9494B0
:10BD40009493600008F8008080800000203F21006C
:10BD500000203F2000809898000000000020203F35
:10BD600020200000000000809898000000C0808023
:10BD7000807F000008F8000080808000203F2402BF
:10BD80002D302000000808F8000000000020203FAF
:10BD9000202000008080808080808000203F200064
:10BDA0003F20003F8080008080800000203F2100F5
:10BDB00000203F200000808080800000001F2020A5
:10BDC00020201F00808000808000000080FFA120D4
:10BDD00020110E000000008080808000000E1120E5
:10BDE00020A0FF80808080008080800020203F2174
:10BDF0002000010000008080808080000033242427
:10BE000024241900008080E0808000000000001FD2
:10BE1000202000008080000000808000001F202083
:10BE200020103F20808080000080808000010E3044
:10BE30000806010080800080008080800F300C03A5
:10BE40000C300F0000808000808080000020312EA8
:10BE50000E312000808080000080808080818E7084
:10BE60001806010000808080808080000021302C36
:10BE70002221300000000000807C0202000000004F
:10BE8000003F404000000000FF00000000000000F4
:10BE9000FF0000000002027C800000000040403FE4
:10BEA000000000000006010102020404000000007E
:10BEB0000000000060010000010000002000000000
:10BEC00020000000002C0000200000000306010BF1
:10BED0000405020925262734350000010001000C65
:10BEE000000100000040000000000200000004000B
:10BEF0000000080000001000445B0020445C0020AB
:10BF0000445D0020446900200B0000000C0000008C
:10BF10000D0000000E0000000F00000010000000E7
:10BF20001100000038000000390000003A00000055
:10BF30003B0000003B000000000102030405060076
:10BF400004000000080000001000000020000000B5
:10BF5000400000008000000000010000010002001D
:10BF600004000800100020004000800000010002D2
:10BF700000040008001000200040008000010203BF
:10BF80000405060708090A0B0C0D0E0F010000003E
:10BF90000200000004000000080000001000000083
:10BFA00020000000400000008000000000010000B0
:10BFB0000002000000040000000800000010000063
:10BFC0000020000000400000008000000607080973
:10BFD0000A171717171728282828282800030306E8
:10BFE00001040602050003051F1C1F1E1F1E1F1F44
:10BFF0001E1F1E1F1C1D1E323637000001000000D0
:10C000000200000004000000080000001000000012
:10C01000200000000000000000000000303132333A
:10C02000343536373839414243444546403058006C
:10C03000303132333435363738396162636465669E
:10C0400040307800040000080000000000000002FA
:10C05000000100001000000004FA97999999D93F57
:10C06000AF788E1DC571CC3F9FC678D0099AC33F6B
:10C07000935555555555E53F599322942449D23F40
:10C08000DE03CB966446C73F44523EDF12F1C23F07
:10C090000000000000000000303132333435363704
:10C0A00038396162636465667870003031323334E8
:10C0B0003536373839414243444546585000000030
:10C0C00002400000000000A0000000000540000049
:10C0D000000000C8000000000C4000000000409C70
:10C0E00000000000194000000020BCBE000000005D
:10C0F00034400000BFC91B8E00000004B5400000A2
:10C10000504BCFD06607E2CF010000006C41000029
:10C110003E8251AADFEEA73401000000D9420000A0
:10C12000DCB5A0E23A301F97FFFFFFFFB4450000E7
:10C13000FD25A0C8E9A3C14FFFFFFFFFFF3F00009F
:10C140000000008000000000FF3F000000000080B1
:10C15000000000000D0A2A2A2A2A2A2A2A2A2A2A24
:10C160002A2A2A2A2A2A2A2A2A2A2A2A2A2A2A2A2F
:10C170002A2A2A2A2A2A2A2A2A2A2A2A2A2A2A2A1F
:10C180002A2A2A2A2A2A2A2A2A2A2A2A2A2A2A2A0F
:10C190002A2A2A2A00000000415445300D0A0000D6
:10C1A00041542B4342430D0A0000000041542B51DF
:10C1B000504F57440D0A000041542B474D520D0A71
:10C1C0000000000041540D0A0000000041542656B2
:10C1D0000D0A0000415426570D0A0000453A20314F
:10C1E000000000002B434243000000004F4B0000C2
:10C1F000504F574552454420444F574E00000000D1
:10C200004552524F5200000041542B51494353476D
:10C21000503D25642C312C222573222C22222C22E5
:10C22000222C310D0A00000041542B435245473D5A
:10C23000320D0A0041542B43475245473D320D0A07
:10C240000000000041542B435245473F0D0A0000B7
:10C2500041542B43475245473F0D0A0041542B514F
:10C26000494143543F0D0A0041542B514343494433
:10C270000D0A000041542B514E57494E464F0D0AAE
:10C280000000000041542B4353510D0A00000000F0
:10C2900041542B514944454143543D25640D0A0006
:10C2A00041542B51494143543D25640D0A0000007F
:10C2B0002B435245473A00002B43475245473A002B
:10C2C0002B514E57494E464F3A0000002B435351D5
:10C2D0003A0000002B51494143543A002B5143434B
:10C2E0004944000041542B5149434C4F53453D258F
:10C2F000642C31300D0A000041542B51494F5045F8
:10C300004E3D312C25642C22544350222C2225737F
:10C31000222C25642C25642C310D0A0041542B510C
:10C320004953544154453D312C25640D0A00000009
:10C3300041542B514953454E443D25642C25640DF1
:10C340000A0000002B514953544154453A00000063
:10C350002B51494F50454E3A000000003E0000006E
:10C3600053454E44204F4B002573000041542B5140
:10C370004654504346473D226163636F756E742295
:10C380002C222573222C222573220D0A0000000086
:10C3900041542B5146545052454E414D453D222566
:10C3A00073222C222573220D0A00000041542B51C8
:10C3B0004654504357443D222573220D0A00000085
:10C3C00041542B5146545053495A453D222573221E
:10C3D0000D0A000041542B514654504E4C53543DCD
:10C3E000222573220D0A000041542B51465450500F
:10C3F00057440D0A0000000041542B51465450434D
:10C400004C4F53450D0A000041542B514654504C9B
:10C41000454E0D0A0000000041542B514654505324
:10C420005441540D0A00000041542B5146545043CE
:10C4300046473D22636F6E746578746964222C25CB
:10C44000640D0A0041542B514654504346473D2247
:10C450007472616E736D6F6465222C25640D0A0021
:10C4600041542B514654504346473D2266696C6502
:10C4700074797065222C25640D0A000041542B51FB
:10C480004654504F50454E3D222573222C25640DB5
:10C490000A00000041542B514654504346473D2268
:10C4A00072737074696D656F7574222C25640D0A42
:10C4B0000000000041542B514654504745543D2242
:10C4C0002573222C22434F4D3A222C25642C2564BF
:10C4D0000D0A00002B514654505057443A2030006A
:10C4E0002B5146545052454E414D453A20300000A4
:10C4F0002B5146545053495A453A20300000000011
:10C500002B51465450535441543A203000000000FF
:10C510000D0A4F4B0D0A0D0A2B51465450474554F6
:10C520003A2030002B514654504E4C53543A203050
:10C53000000000002B514654504357443A20302C01
:10C54000300000002B51465450434C4F53450000DF
:10C550002B4F4B00A0C6000800000020F40600008E
:10C560006C010008F4C80008F40600207C95000067
:10C57000C80100081001000043000000F8FFFFFFA1
:10C5800000404040404040404040414141414140E6
:10C59000404040404040404040404040404040409B
:10C5A000400502020202020202020202020202022A
:10C5B000022020202020202020202002020202022F
:10C5C0000202909090909090101010101010101087
:10C5D0001010101010101010101010100202020293
:10C5E00002028888888888880808080808080808D7
:10C5F00008080808080808080808080802020202D3
:10C6000040000000000000000000000000000000EA
:10C61000000000000000000000000000000000001A
:10C62000000000000000000000000000000000000A
:10C6300000000000000000000000000000000000FA
:10C6400000000000000000000000000000000000EA
:10C6500000000000000000000000000000000000DA
:10C6600000000000000000000000000000000000CA
:10C6700000000000000000000000000000000000BA
:10C68000000000001C00000043000000F8FFFFFF56
:10C690000C0000000E0000000F0000002E00000043
:10C6A00021057D0341424D000E7453686F70333491
:10C6B000343739343734393010015A3132312E356C
:10C6C0002E3231372E3235321215057C2F41424D34
:10C6D0002230E995110510581B701713ACC12408BE
:10C6E0008A021AF0081AFF011112C21B0804103244
:10C6F000011AC414320AAAEC1C2203191F111ACC05
:10C7000014190B114BF8C41C1ADC101A0435291427
:10C710005A981CB938193532040A15D41C32050A46
:10C7200015B81C32065AA08CDAE41C411A680C2990
:10C73000401ADC08A9A829C41A280C091254293B5C
:10C740005A441CAAB038191929140A15343829C4B6
:10C750005A501CDAB83829845A741CAAC01C19898A
:10C7600029C45A841CDACC3832070A1508702A0802
:10C77000FC190C1ADC5DB91C195432091A900C1AF8
:10C78000900CE91C320A5A5C54DAD470411AF80C45
:10C790002AC8CCCAC3381903111AE40C0A11648CD4
:10C7A000293B1A1C3029E8AA4438191929681A307B
:10C7B000142A1478D95432045A681CDA601C4113C4
:10C7C00028C42A08B0E970291F1A6C3009121C29E4
:10C7D0008C0A156038298C0A15441C298C0A15947A
:10C7E0001C29D81A7C1C0A11C81C32065A18381188
:10C7F000CAC51C32075AACA8DA341C32085AE81CE5
:10C800001AD440A91C2A0914591CDA243829145AAC
:10C81000C01CDAF038320B1AB4143228AA103822AD
:10C8200001320C5A08A8DA5054320D1A90543214BE
:10C83000DAE054320E5AF81CDA443813E1341408A2
:10C8400013351408402C3220146840581A2009E28D
:10C8500068180801020209020A0A8110090102038C
:10C860000A030B0B0214380140124412401A480408
:10C870001A4C0412501B4004141A04141A04141AFB
:10C88000041413833D1B088D041A97041AA1044154
:10C8900012081C02401C041A30041A44041A5804DA
:10C8A0001A6C041A800419911B401C041A30041AD3
:10C8B00044041A5804111A08681A0C041A10041AAD
:10C8C00014041A18041A1C041A2004011612401A1F
:10C8D00004041A08041A0C041A100412143D40022D
:10C8E00004068019C02A040415060708098CA24A08
:04C8F00004E2491401
:04000005080002C12C
:00000001FF
